:1070560000001D0200000301FA0400EF0500030A08
:107066000A5A0B001E0C00FA0D00030E00040F0155
:1070760064100096120132130AFA14010217010A6B
:107086001801EF1905321A010A1B01EF1C05321F00
:10709600FFFF20FFFF23011E2400642A00FA2B00B5
:1070A600FA2C50782D003D2E004630006432507880
:1070B6003300003432FA3501643601643701503842
:1070C6000A643A00033B00043C00643E003C3F0077
:1070D6000140FFFF411450420A5A430AC844053290
:1070E6004500B44600FA4900024B00014C00FA5034
:1070F6000404510596520A32530B46540A96570514
:1071060046590A465A32FA5B010A5C0A325E000A9E
:107116005F00646200FE64010567FFFF68010169A4
:1071260001016A05966B00006C32966D00047300CF
:10713600017400017801327901327E0064810064B5
:1071460084FFFF8800028A00019D0A969E00019F27
:10715600FFFFA0010CA2000AA3FFFFA4FFFFA5FFEB
:10716600FFA6FFFFA7FFFFA8FFFFA9FFFF0101186A
:107176001500022F003C4701184803045601044E2F
:10718600FFFF58000261FFFF6600028500AF860020
:10719600018700FA89010A990008A100FAFAFAFAA9
:1071A60001010C1500022F1E3C4701184803045626
:1071B60001034EFFFF58000261FFFF6600028500D3
:1071C600AF8600018700FA89010A990000A1000034
:1071D600FAFAFA01010C1500002F1E3C47010C4873
:1071E60003035601014EFFFF58000061FFFF6600D2
:1071F6000085FFFF86FFFF87FFFF890102990000D8
:10720600A10000FAFAFA0065006F00790083008D8C
:10721600009700A100AC00B600C000CA00D400DE92
:1072260000E800F2005800600068007000780080F6
:1072360000880090009800A000A800B000B800C127
:1072460000C800D000D800DF00E600EE00F60041DE
:107256000047004D00530059005F0065006C007147
:107266000077007D00830089008F0095009B00A2B7
:1072760000A700AC00B200B900C000C500CA00D229
:0A72860000D500DD00E100E700EF95
:103CD80085F97385FA747E017F00E5741273A2E595
:103CE800732FFF50010E8E598F5A900014E0FCA3D9
:103CF800E0FDEF2DFDEE3CFC8C5B8D5C900034E02C
:103D0800FAA3E0FBED2BFBEC3AFA8A5B8B5C22759D
:103D1800A71085F97385FA747E017F00E574127324
:103D2800A2E5732FFF50010E8E598F5A9000E4E0E0
:103D3800B40210AC2CAD2DEF2DFDEE3CFC8C5B8D50
:103D48005C8016AE59AF5A900014E0FCA3E0FDEF7A
:103D58002DFDEE3CFC8C5B8D5CAE5BAF5C90003463
:103D6800E0FCA3E0FDEF2DFDEE3CFC8C5B8D5C22BE
:103D7800E55CF5FBE55BF5FCD29322E55CF5E9E54E
:103D88005BF5EAD29422E55CF5EBE55BF5ECD291C4
:103D980022E55CF5EDE55BF5EED2922275A710E51C
:103DA8005CF5FBE55BF5FC75A700D2872275A710CB
:103DB800E55CF5E9E55BF5EA75A700D2902275A701
:103DC80010E55CF5EBE55BF5EC75A700E5B544108F
:103DD800F5B52275A710E55CF5EDE55BF5EE75A781
:103DE80000E5B54420F5B522E50C906C09F82828C3
:103DF80073023EB675E700A237B34008E5B544083C
:103E0800F5B58006E5B554F7F5B575E710023EB689
:103E180075E700A237B34008E5B54402F5B580065A
:103E2800E5B554FDF5B575E710023EB6A23792A286
:103E3800807CA23792A1807675E700A237B340084C
:103E4800E5B54440F5B58006E5B554BFF5B575E769
:103E580010805B75E700A237B34008E5B54480F5EC
:103E6800B58006E5B5547FF5B575E7108040A237F3
:103E78009287803AA2379290803475E700A237B3D0
:103E88004008E5B54410F5B58006E5B554EFF5B53D
:103E980075E710801975E700A237B34008E5B54407
:0E3EA80020F5B58006E5B554DFF5B575E710D9
:106C0900023DF9023DFC023E18023E34023E3A02C0
:106C19003E40023E5B023E76023E7C023E82023EDE
:016C29009DCD
:103EB600227431900155F07432900156F0742D90B1
:103EC6000157F07431900158F07420900159F07444
:103ED6003490015AF0744390015BF0747990015C60
:103EE600F0746C90015DF0742090015EF074209087
:103EF600015FF07420900160F07420900161F0740D
:103F060020900162F07420900163F02290088CE00A
:103F1600FEA3E0FF741DD39F74019E400C90705663
:103F2600120048E493F599804C90F802E493B405A6
:103F36001490088CE0FEA3E0FF907089120048E41C
:103F460093F599803090F802E493D3940540149049
:103F5600088CE0FEA3E0FF907056120048E493F54B
:103F660099801290088CE0FEA3E0FF9070BC1200CE
:103F760048E493F59990088C1273B090088CE0FE93
:103F8600A3E0FFEFB45007EEB40103754D0022AE77
:103F960059AF5A741E8E048F05FF1273928C5B8D77
:103FA6005CAE59AF5A741E8E048F05FF1273BD8C1A
:103FB600598D5AC200E55A45596013741EC3955A65
:103FC600FFE49559FE8E598F5A785B1273F5E573A7
:103FD600A85BB80015D3955C4010E573C3955CFFEC
:103FE600E4955BFE8E5B8F5C8012E573240CC395B3
:103FF6005CFFE4955BFE8E5B8F5CD200AE5BAF5CD4
:10400600740C6F4E700B755C0B755B0075730180DD
:104016000375730022900092E0B40104C207800287
:10402600D207900093E0B40104C2088002D208903F
:1040360000D0E075F0D7A4FFAEF0740A8E048F05A9
:10404600FF127392900880ECF0A3EDF09000D0E0A0
:1040560075F02BA4FFAEF0900010EEF0A3EFF07E0B
:10406600017F0090008EE01273A29000D1E08E04D2
:104076008F05FF127392740AFF1273928D6090007F
:10408600DAE075F0D7A4FFAEF0740A8E048F05FF50
:10409600127392900884ECF0A3EDF09000DCE060DF
:1040A600139000DCE0F5F0741684FF7E00EF9008B4
:1040B600E2F0800674649008E2F09000D2E090008E
:1040C6006CF090011EE0900079F0900120E0FE90E7
:1040D60000CEE08E0088F0A4FFAEF0EF9008EBF083
:1040E6009000F9E075F013A4FDACF0900034ECF00C
:1040F600A3EDF0A221B3401690016AE0700C900186
:104106006BE0700690016CE060028002C2219001B3
:104116006AE0B4300F90016BE0B4470890016CE0A0
:10412600643B60028004D2228002C22274E39000C3
:104136006BF09000BBE0B40B0874E390006BF0806A
:104146005A9000BBE0B419129000D1E09071F712BA
:10415600008CE49390006BF080419000BBE0B41EAD
:10416600129000D1E090721512008CE49390006BCF
:10417600F080289000BBE0B428129000D1E0907245
:104186003F12008CE49390006BF0800F9000BBE030
:10419600B446089000B2E090006BF090008BE0FE11
:1041A6009008ECE06E601A7599E612019C74AB906B
:1041B6000045F012069A7509647508001205E48038
:1041C600FE900083E0700674009000B8F0900070D6
:1041D600E0FE9000B8E0B50663900073E0FE900044
:1041E600D6E0B50657900071E0FE9000E4E0B50613
:1041F6004B900077E0FE90008BE0B5063F90007490
:10420600E0FE9000C6E0B50633900072E0FE900036
:10421600D4E0B50627900075E0FE9000F1E0B50603
:104226001B900076E0FE9000F2E0B5060F90007855
:10423600E0FE900104E06E70030244B3900093E048
:1042460070089000D4E06404600280067403900055
:10425600D4F090004DE0C394055008740290010715
:10426600F080149000E4E060087406900107F08086
:1042760006740A900107F090008BE0B40106740002
:1042860090008BF090008BE0B4020674009000D68C
:10429600F090008BE0B4030674009000E3F0900009
:1042A600D6E0D394014027741B900109F074009066
:1042B60006D4F074009006D5F074009000A0F0903B
:1042C60000B8E0B4020674019000B8F080339000A4
:1042D600B8E0B4021A7400900109F074009006D494
:1042E600F074009006D5F0741B9000A0F080127454
:1042F60000900109F0741B9006D4F074009000A0A1
:10430600F09000B8E06014741C90009FF074009068
:1043160006D8F074009006D9F0800C740090009FC7
:10432600F0741C9006D8F09000F1E06014741990B7
:10433600010BF074009006CCF074009006CDF0806E
:104346000C740090010BF074199006CCF09000F2FA
:10435600E06014741A90010CF074009006D0F074AA
:10436600009006D1F0800C740090010CF0741A9045
:1043760006D0F0900104E06014742A90077CF07473
:10438600009006C8F074009006C9F0800C74009086
:10439600077CF0742A9006C8F09000E4E07032744E
:1043A600059006DCF074069006E0F074079006E4CB
:1043B600F074089006E8F07400900778F0740090A6
:1043C6000779F0740090077AF0740090077BF0800C
:1043D6004874009006DCF074009006DDF0740090DE
:1043E60006E0F074009006E1F074009006E4F074C4
:1043F600009006E5F074009006E8F074009006E977
:10440600F07405900778F07406900779F0740790B9
:10441600077AF0740890077BF09000D4E0D39402FA
:10442600401A741590076CF0741690076DF07417A7
:1044360090076EF0741890076FF080277415900738
:104446006CF09000D4E0B40208741690076DF0800A
:1044560006740090076DF0740090076EF07400907B
:10446600076FF0D2209000B8E0900070F09000E462
:10447600E0900071F09000D6E0900073F09000C6D6
:10448600E0900074F09000D4E0900072F090008B01
:10449600E0900077F09000F1E0900075F09000F267
:1044A600E0900076F0900104E0900078F09000EE45
:1044B600E0B40117900020740FF0A374FFF0900091
:1044C60022E4F0A3F074029000EEF09000EEE0B467
:1044D6000341900022E0FEA3E0FF900020E0FCA351
:1044E600E0FD1273ED74101273A27408120039EF16
:1044F6009000EDF0EF700674FF9000EDF074009000
:1045060000EEF0900021E09000A4F0900020E090F2
:1045160000A5F090007FE090007CF090007EE09097
:10452600007BF09000ADE0C3941E50569000ADE0C5
:10453600F404241E90007DF090007DE075F01E844A
:10454600FF7E008F7390007DE075F01E84ADF07CD9
:10455600008D7490007BE0D39574400D90007BE055
:10456600C3957490007BF0800F90007BE0241EC3FF
:10457600957490007BF0057390007CE025739000A5
:104586007CF090007CE090003EF090003EE0240637
:1045960090003FF090003EE0D39418400B90003E10
:1045A600E0C3941890003EF090003FE0D39418408A
:1045B6000B90003FE0C3941890003FF0C224900097
:1045C6003EE0D3940C400D90003EE0C3940C900066
:1045D6003EF0D224C22590003FE0D3940C400D90CB
:1045E600003FE0C3940C90003FF0D225900042E4D7
:1045F600F090003EE0B40C0C9000427401F0900084
:104606003E7401F0900043E4F090003FE0B40C0CDF
:104616009000437401F090003F7401F090007FE039
:10462600FE9000E2E02E900046F0900046E0D39423
:104636000C400B900046E0C3940C900046F09000AE
:1046460046E0D3940C400B900046E0C3940C9000D7
:1046560046F0900046E064066007900046E0B40C21
:1046660006900046E004F0900046E0D3940C400B20
:10467600900046E0C3940C900046F0900046E0D3CC
:104686009406400D900046E0C39406900047F080E3
:104696000A900046E02406900047F0755D069000FB
:1046A6007FE0FE9000C5E0D39E501390007FE0FEB1
:1046B6009000C5E0F4042E04900040F080139000B2
:1046C6007FE02418FE9000C5E0F4042E049000401C
:1046D600F0900040E075F00684AFF07E00EF4E707B
:1046E60006900040E004F0900040E0B41906900007
:1046F600407401F0900040E0D3940C400F900040CD
:10470600E0C3940C900040F0D21B8002C21B9000C4
:1047160040E0D39406400D900040E0C3940690001C
:1047260041F0800A900040E02406900041F012011A
:104736009C22C293C294C291C292C287C290E5B52E
:1047460054EFF5B5E5B554DFF5B5C296C295C2A0EE
:10475600C297C2A2C2A1E5B554BFF5B5E5B5547F6F
:10476600F5B5E5B554FBF5B5C209755E469000C8CA
:10477600E07005756D028003756D03755400755301
:104786000090000874FFF0A374DCF0C20EC211742E
:10479600C8900036F074C890003AF0755200755112
:1047A60000C204754600E56FB41303756F007563A8
:1047B60000900016E4F0A3F0757010C20CC20DC292
:1047C6000375560075550090000AE4F0A3F09000BA
:1047D6000CE4F0A3F0C22775580075570090008AC4
:1047E600E075F032A4FFAEF090001EEEF0A3EFF0FD
:1047F60090007AE4F09008E8E4F0C223D218C217D9
:10480600D219C21AC21BC21C90000EE4F0A3F022F9
:10481600755A00755900AE59AF5A741CC39F74017E
:104826009E500302490A907056120048E493645F52
:104836006023907056120048E493647E601790706F
:1048460056120048E4936481600B9070561200483B
:10485600E493B484030248EAAE59AF5A90705612F4
:104866000048E49390007E1273D30FBF00010EE060
:10487600FC907056120048ECFEE493FFEEC39F5086
:1048860026AE59AF5A0FBF00010E9070561200485F
:10489600AE59AF5AE493FC907056120048E49390D8
:1048A600007E1273D3ECF0AE59AF5A9070561200D8
:1048B60048E49390007E1273D3E0FC907058120087
:1048C60048ECFCE493FDECD39D401990705812001F
:1048D60048E493FC907056120048E49390007E12D0
:1048E60073D3ECF0AE59AF5A74022FFF50010E8EFF
:1048F600598F5A785A740126F6500418E436F64051
:104906000302481C22755A00755900AE59AF5A74F5
:1049160032BE00039F50030249D8907173120048BB
:10492600E49390007E1273D30FBF00010EE0FC905B
:104936007173120048ECFEE493FFEEC39F5026AE5F
:1049460059AF5A0FBF00010E907173120048AE594D
:10495600AF5AE493FC907173120048E49390007E82
:104966001273D3ECF0AE59AF5A907173120048E44B
:104976009390007E1273D3E0FC907175120048ECA0
:10498600FCE493FDECD39D4019907175120048E448
:1049960093FC907173120048E49390007E1273D3D7
:1049A600ECF0AE59AF5A742D6F4E7006755A3375CA
:1049B6005900AE59AF5A74022FFF50010E8E598F0F
:1049C6005A785A740126F6500418E436F640030263
:1049D600491122755A00755900AE59AF5A7432BE44
:1049E60000039F5003024AA69071A6120048E49362
:1049F60090007E1273D30FBF00010EE0FC9071A6EB
:104A0600120048ECFEE493FFEEC39F5026AE59AF6A
:104A16005A0FBF00010E9071A6120048AE59AF5A48
:104A2600E493FC9071A6120048E49390007E127302
:104A3600D3ECF0AE59AF5A9071A6120048E49390A9
:104A4600007E1273D3E0FC9071A8120048ECFCE4DF
:104A560093FDECD39D40199071A8120048E493FC95
:104A66009071A6120048E49390007E1273D3ECF086
:104A7600AE59AF5A742D6F4E7006755A337559007C
:104A8600AE59AF5A74022FFF50010E8E598F5A78C5
:104A96005A740126F6500418E436F640030249DF3C
:104AA60022755A00755900AE59AF5A7432BE0003CA
:104AB6009F5003024B749071D9120048E493900002
:104AC6007E1273D30FBF00010EE0FC9071D9120065
:104AD60048ECFEE493FFEEC39F5026AE59AF5A0F43
:104AE600BF00010E9071D9120048AE59AF5AE49337
:104AF600FC9071D9120048E49390007E1273D3ECB7
:104B0600F0AE59AF5A9071D9120048E49390007EE6
:104B16001273D3E0FC9071DB120048ECFCE493FDC9
:104B2600ECD39D40199071DB120048E493FC907120
:104B3600D9120048E49390007E1273D3ECF0AE597C
:104B4600AF5A742D6F4E7006755A33755900AE59AB
:104B5600AF5A74022FFF50010E8E598F5A785A742D
:104B66000126F6500418E436F64003024AAD2285C3
:104B7600F97385FA747E017F00E5741273A2E573FA
:104B86002FFF50010E8E598F5AAC5BAD5CEF2DFD99
:104B9600EE3CFC8C5B8D5CD293D294D291D292E5A2
:104BA6005CF5FBE55BF5FCE55CF5E9E55BF5EAE55F
:104BB6005CF5EBE55BF5ECE55CF5EDE55BF5EE222A
:104BC60075A71085F97385FA747E017F00E5741266
:104BD60073A2E5732FFF50010E8E598F5A7E017F07
:104BE60076900103E01273A2AC59AD5AED2FFFEC9B
:104BF6003EFE8E5B8F5CE55CF5FDE55BF5FE9000A9
:104C06006CE4F075A7007412900049F02285F973E0
:104C160085FA747E017F00E5741273A2E5732FFF97
:104C260050010E8E598F5A900010E0FCA3E0FDEF64
:104C36002DFDEE3CFC8C5B8D5CE55CF5FDE55BF5E6
:104C4600FE22056422A2D8B34002C293A2D9B34081
:104C560002C294A2DAB34002C291A2DBB34002C2FE
:104C660092A2DCB34030A29650067419900049F027
:104C7600A29550067419900049F0A2A05006741926
:104C8600900049F0A29750067419900049F0C29618
:104C9600C295C2A0C29775D8402285A77275A71083
:104CA600A2D8B34002C287A2D9B34002C290A2DA08
:104CB600B34006E5B554EFF5B5A2DBB34006E5B55E
:104CC60054DFF5B5A2DCB340089000D2E090006C4A
:104CD600F075D8408572A72290F800E493640660C8
:104CE6000280FE12009E75A70075D80075D904755E
:104CF600DA0975DB0975DC0975DD0975DE0975D814
:104D06004075A71075D80075D90475DA0975DB09E1
:104D160075DC0975DD0975DE0975D84075A70012C1
:104D260000FB7509C87508001205E475A70FE5FCB8
:104D3600900058F0E5FB900059F0E5FA90005AF023
:104D4600E5F990005BF075A70090F800E493F5276D
:104D5600120703900895E0D394035007900895E056
:104D6600B401067400900895F0900895E09008EC60
:104D7600F074019000C7F0900895E0906C2AF8282E
:104D86002873802A802875A70F75F30F75A700A2D0
:104D9600A3400674029000C7F0801375A70F75F341
:0E4DA6001775A700A2A4400674029000C7F083
:0C6C2A00024D88024D8A024D8C024DA1E3
:104DB4009000C7E0B4022AC216120AAC7402900032
:104DC400C7F0900895E0906C36F82828738010801E
:0F4DD4000E74009000D6F0800674009000E3F09B
:0C6C3600024DD1024DD3024DD5024DDDC0
:104DE3008028D2161209C174019000C7F09008956B
:104DF300E0906C42F82828738010800E74009000B5
:0A4E0300D6F0800674009000E3F082
:0C6C4200024DFB024DFD024DFF024E070B
:104E0D0090F807E493900065F0900065E0440890F9
:104E1D000065F0900065E054FE900065F012039D72
:104E2D00123EB79008A2E090016AF09008A3E090BE
:104E3D00016BF09008A4E090016CF090016AE070B5
:104E4D000C90016BE0700690016CE060028004C272
:104E5D00218002D2219000B8E004900070F0124839
:104E6D001690F802E493B405051249D9801290F812
:104E7D0002E493D39405400512490B8003124AA70F
:104E8D0074009000EEF012401BE5B54401F5B574C9
:104E9D000690004BF0740090004CF0740190004DA2
:104EAD00F090F802E49390004EF090F803E49390A4
:104EBD00004FF090F804E493900050F074069000C9
:104ECD0051F090004EE0B405067405900051F0903D
:104EDD00004EE0B404067404900051F07407900085
:104EED0052F07403900053F07406900054F0740760
:104EFD00900055F090F805E493900056F090F80668
:104F0D00E493900057F0740090005FF074009000EF
:104F1D0060F07400900061F07400900062F0740015
:104F2D00900063F07400900064F074FF900066F0E0
:104F3D00A2B6B39205A2B3B39206A2A4B3921EA2D7
:104F4D00A3B3921F900067E4F0756F00743A900759
:104F5D007EF074FD90077FF0900068E4F0756E01AF
:104F6D00900049E4F09000C8E0B40106741A900076
:104F7D0049F0C21D756300C20AD20BC203757100E0
:104F8D00C220120586755F00756B00756100756531
:104F9D0032756600756700756800756900756A0081
:104FAD00900016E4F0A3F0756C00D2B2D2A4D2B08A
:104FBD00D2B1D2A3D2A7D2A6D2A5D2B77E017F00FD
:104FCD009000A5E01273A29000A4E02FFF50010EF7
:104FDD00900020EEF0A3EFF0EFD394FFEE940F408E
:104FED0007900020E4F0A3F09000EDE0700674FF50
:104FFD009000EDF09000C8E07005756D02800375AE
:10500D006D03740090010AF0740090010DF07400AE
:10501D0090010EF074299006C4F07401900774F09D
:10502D007402900775F07403900776F0740490077E
:10503D0077F07400900770F07400900771F07400B1
:10504D00900772F07400900773F0D29CE570D394C2
:10505D001040037570109006C5E0D3940C40067493
:10506D00009006C5F09006C9E0D3940C400674007C
:10507D009006C9F09006CDE0D3940C4006740090D4
:10508D0006CDF09006D1E0D3940C40067400900646
:10509D00D1F09006D5E0D3940C400674009006D55F
:1050AD00F09006D9E0D3940C400674009006D9F028
:1050BD009006DDE0D3940C400674009006DDF09070
:1050CD0006E1E0D3940C400674009006E1F09006E2
:1050DD00E5E0D3940C400674009006E5F09006E9E7
:1050ED00E0D3940C400674009006E9F0D2EC75CF35
:1050FD0001A298B34005C298120C14E54D6006A2AA
:10510D0099B3B340028005C2991210A3E54E640114
:10511D006005E54EB4040280D5C28E7E107F00E599
:10512D00641273A2E58D75F010A4FDACF0EF2DFDAA
:10513D00EE3CFCE58B75F01084FF7E00ED2FFFEC4F
:10514D003EFE8E538F54D28E9000ABE060099000DE
:10515D00ABE0C3943D4002805C9000181273B09098
:10516D000018E0FEA3E0FF90001AE0FCA3E0FDEFC5
:10517D00B50542EEB5043EB214A204B3401975E76D
:10518D0000A214B34008E5B54404F5B58006E5B5B5
:10519D0054FBF5B575E71090001AE0FEA3E0FF9003
:1051AD00001CE0FCA3E0FDEF2DFDEE3CFC90001A91
:1051BD00ECF0A3EDF09000B8E060099000B8E0C30A
:1051CD009403400302527F122FCEA2044008900098
:1051DD00A2E0F545801BE55FC39560500575450060
:1051ED00800F90008FE0C3956150069000B5E0F5FB
:1051FD0045E54575F002A4FFAEF090088AEEF0A3E8
:10520D00EFF075E700AC2EAD2FEDD39FEC9E402C4B
:10521D00E5B5547FF5B59006C5E07006E5B554F7D4
:10522D00F5B59000B8E0B402099000D6E0C3940241
:10523D0040028006E5B54440F5B58033900067E047
:10524D00C39441502AE5B54480F5B59006C5E0708C
:10525D0006E5B54408F5B59000B8E0B40209900034
:10526D00D6E0C3940240028006E5B554BFF5B5758E
:10527D00E7109000B8E0B4032A1230E975E700AEEC
:10528D002EAF2F90088AE0FCA3E0FDEFD39DEE9C9E
:10529D004008E5B54480F5B58006E5B5547FF5B514
:1052AD0075E710900093E06009A2B3300601B3B327
:1052BD0040028056A2B3300601B3404EA2B330086F
:1052CD0001B34039A2184030900079E0D3955E408B
:1052DD00259008E8E0701390007AE0B4010690087C
:1052ED00E87401F090007AE004F0A217B340059045
:1052FD00007AE4F0D217D218A208B39206A208B32E
:10530D0030B301B34004A2089206A2B6300501B332
:10531D005003025A26A2B6300501B35003025A2695
:10532D00A2B6300701B35003025938756E009000D4
:10533D00ABE0B43D1975E700A207B34008E5B554DD
:10534D00FBF5B58006E5B54404F5B575E710055ECA
:10535D00A209B3B35013AE53AF54900008E0FCA3B1
:10536D00E0FDEDC39FEC9E400302553DE56DB4039A
:10537D002EA227B34022E55EB40C03756D01E55EE8
:10538D00C3940C50069000497401F0E55ED3940C63
:10539D0040067402900049F0755E01D2278062E5E7
:1053AD006DB4020A756D01755E0CC217C219E55E0A
:1053BD00B40C05755E018049900049E07034E55EDE
:1053CD00C3940C50069000497401F0E55ED3940C23
:1053DD0040067402900049F0E55EC3940C5002D271
:1053ED001DE55ED3940C4002D21DC296C295C2A09B
:1053FD00C2979000C8E0B401051247388003755E6E
:10540D0001AE55AF56AC53AD54EF2DFDEE3CFC74D3
:10541D0003FF1273928C558D569000ABE06009908E
:10542D0000ABE0C3943D40028049900018E0FEA31C
:10543D00E0FF9000ABE08E048F05FF1273927401B4
:10544D008C068D0712003990001CEEF0A3EFF09042
:10545D00001CE0F8A3E090001AC8F0A3C8F090007B
:10546D0018E4F0A3F0C21475E700E5B554FBF5B5EB
:10547D0075E710A2A4B34002C21EA2A3B34002C29C
:10548D001FA21DB34002C21DB21A9008E8E0B4017C
:10549D0011A217B34004D21A8002C21A74029008E6
:1054AD00E8F09008E8E0C394025006A204B3B340BC
:1054BD0002800674029008E8F09000D4E064046065
:1054CD00079000C6E0B40462900093E06006900877
:1054DD00E8E07002800DA219301701B3400590006D
:1054ED007AE4F09000C8E064016006A223B3B350E3
:1054FD0017900093E06009A217301901B3B3400271
:10550D0080067405900049F0B219A218B3401BA291
:10551D0017B34004D2198002C2199000C8E070067A
:10552D009008E8E070028002D223C217C218803AB8
:10553D00AE55AF56AC53AD54EF2DFDEE3CFC7401A2
:10554D008C068D071200398E558F56E56DC394026A
:10555D00500DAC53AD547498C39D743A9C40028069
:10556D00091247387406900049F0E55EB40C1274C8
:10557D0003900049F0D21D9000C8E0B4010312471A
:10558D0038AE57AF58AC53AD54EF2DFDEE3CFC8CFF
:10559D00578D58AE53AF54EFD39DEE9C40119000F4
:1055AD000EE0FAA3E0FBEBC394E8EA94034002801B
:1055BD000690000E1273B090000CE0FEA3E0FFAC5D
:1055CD0053AD54EF2DFDEE3CFC90000CECF0A3ED33
:1055DD00F09000C8E0B4011DAE53AF5474051273C2
:1055ED00A274038E048F05FF127392900008ECF0E5
:1055FD00A3EDF08016AE53AF5474031273A2740171
:10560D00120039900008EEF0A3EFF0C28E758D00F8
:10561D00758B00756400755401755300D28EE55E6F
:10562D00240275F00384AFF07E00EF4E6003025646
:10563D00C0E56D6013AE55AF5674031273A29000A2
:10564D000AEEF0A3EFF0800F90000CE0F8A3E090CD
:10565D00000AC8F0A3C8F090000AE0FEA3E0FFEF37
:10566D004E600B7C7C7D101272908E518F5290008B
:10567D000CE4F0A3F0AE51AF527428BE00039F505E
:10568D0010E5632FFF50010E74011200398E518FFA
:10569D00528552639000CFE0A851B8000DD39552BA
:1056AD004008E552900048F080099000CFE014903A
:1056BD000048F09000C6E0B40408900040E0655E3C
:1056CD006002800EA21A301B01B34004D21C80026E
:1056DD00C21CE55E64046005E55EB40A099000B87D
:1056ED00E06003122C84900046E0655E6007900038
:1056FD0047E0B55E03756F00A20A5003025878901B
:10570D0000D4E0C394045006A209B3B3400302577A
:10571D00C3900084E0B40173900106E0B40214124A
:10572D00124490006DE075F0BCA4FFAEF08E5B8F5F
:10573D005C8056E56775F00A84FF7E0090057E1249
:10574D000048E0F55A755900AE59AF5A9000A9E0DE
:10575D001273A274648E048F05FF1273928C5B8D8D
:10576D005CE55C900044F0AE59AF5A900082E012B7
:10577D0073A274648E048F05FF12739274BC8C0631
:10578D008D071273A28E5B8F5C8017900082E0757F
:10579D00F0BCA4FFAEF08E5B8F5C9000A9E0900092
:1057AD0044F0E561C394CC5006E55C455B70028026
:1057BD0003124B75D20A9000D4E0B404069008E8A9
:1057CD00E07003025878900084E0B40173900106F4
:1057DD00E0B4021412124490006DE075F0BCA4FF09
:1057ED00AEF08E5B8F5C8056E56775F00A84FF7EA8
:1057FD000090057E120048E0F55A755900AE59AF7C
:10580D005A9000A9E01273A274648E048F05FF12E2
:10581D0073928C5B8D5CE55C900044F0AE59AF5A91
:10582D00900082E01273A274648E048F05FF1273D0
:10583D009274BC8C068D071273A28E5B8F5C8017E1
:10584D00900082E075F0BCA4FFAEF08E5B8F5C9093
:10585D0000A9E0900044F0E561C394CC5006E55CEE
:10586D00455B70028003124B75D20AE56DB40106DB
:10587D00E55E6404600280189000D4E0B404057500
:10588D007003800975700090004A7401F0756D0009
:10589D00E56D60030259339000CBE0600D90006C14
:1058AD00E0A851B800069552400280389000CBE038
:1058BD00B4021790003EE0655E600790003FE0B5D2
:1058CD005E03757003756C00800CC201756C0090E1
:1058DD000016E4F0A3F090006CE0600674099000EF
:1058ED0049F0804290003EE0655E600790003FE029
:1058FD00B55E339000D4E0B4040FA223B340057518
:10590D0070008003757003800375700090003EE099
:10591D00B55E0690004A7401F090003FE0B55E065A
:10592D00740290004AF0A207B39205A207B330B6F5
:10593D0001B35003025A26756E019000ABE0B43DE1
:10594D001975E700A207B34008E5B54404F5B58025
:10595D0006E5B554FBF5B575E71075E700E5B544FB
:10596D0001F5B575E710742B900067F0A20792054D
:10597D00E55ED394484014D209E55ED39454400BB0
:10598D007404900049F0D21D755E469000D3E0B4CA
:10599D000107E56AC3944140028018E56AC3941477
:1059AD0050087413900049F08006740E900049F071
:1059BD00124738900051E0FE90004EE0C39E400922
:1059CD0090004EE0D39408400974FB900049F0120A
:1059DD00473890004FE0601590004FE0FE90004D6D
:1059ED00E06E600974FC900049F012473890005049
:1059FD00E06015900050E0FE900052E06E6009747A
:105A0D00FE900049F0124738900895E0600690012D
:105A1D0003E060028003120B97A21DB34008C296EB
:105A2D00C295C2A0C297900103E0600CAE51AF5277
:105A3D007414BE00059F4002803790008BE0906C7F
:105A4D004EF8282873802A8028A2A3B35005A21FE0
:105A5D00B340028005124BC6D21F8015A2A4B350CD
:105A6D0005A21EB340028005124BC6D21E800280D5
:015A7D000028
:106C4E00025A52025A54025A56025A69025A7C0287
:026C5E005A7E5C
:105A7E00A20CB3B35008900040E0655E6003025D77
:105A8E0079A202B35006A201B3B34003025D759032
:105A9E0000C6E0B404028003025D519008E8E0B451
:105AAE0002028003025D46A21CB35003025BFF128A
:105ABE003CD8900117E0601F900014E0FEA3E0FFB9
:105ACE0090010FE01273A274C88E048F05FF12733B
:105ADE00928C5B8D5C800A900014E0F55BA3E0F580
:105AEE005CAE5BAF5C745E1273A274058E048F05A0
:105AFE00FF127392AE59AF5AED2FFFEC3EFE8E5B46
:105B0E008F5C900034E0FCA3E0FDEF2DFDEE3CFC3D
:105B1E008C5B8D5C123D78A203B34068123D1790EA
:105B2E000117E0601F900014E0FEA3E0FF90010F4C
:105B3E00E01273A274C88E048F05FF1273928C5BF1
:105B4E008D5C800A900014E0F55BA3E0F55CAE5B23
:105B5E00AF5C745E1273A274058E048F05FF127310
:105B6E0092AE59AF5AED2FFFEC3EFE8E5B8F5C90DE
:105B7E000034E0FCA3E0FDEF2DFDEE3CFC8C5B8DD4
:105B8E005C123DA49000E4E0B40263123D17900154
:105B9E0017E0D39404401BAE2CAF2D900113E012EE
:105BAE0073A274C88E048F05FF1273928C5B8D5C8A
:105BBE008006852C5B852D5CAE5BAF5C745E1273CC
:105BCE00A274058E048F05FF127392AE59AF5AED73
:105BDE002FFFEC3EFE8E5B8F5C900034E0FCA3E06A
:105BEE00FDEF2DFDEE3CFC8C5B8D5C123DA4025D49
:105BFE0044123CD8900117E0D39403401F90001438
:105C0E00E0FEA3E0FF900111E01273A274C88E04AF
:105C1E008F05FF1273928C5B8D5C800A900014E0EE
:105C2E00F55BA3E0F55CAE5BAF5C745E1273A274C1
:105C3E00058E048F05FF127392AE59AF5AED2FFFEA
:105C4E00EC3EFE8E5B8F5C900034E0FCA3E0FDEF3B
:105C5E002DFDEE3CFC8C5B8D5C123D8EA203B340A1
:105C6E006B123D17900117E0D39403401F90001460
:105C7E00E0FEA3E0FF900111E01273A274C88E043F
:105C8E008F05FF1273928C5B8D5C800A900014E07E
:105C9E00F55BA3E0F55CAE5BAF5C745E1273A27451
:105CAE00058E048F05FF127392AE59AF5AED2FFF7A
:105CBE00EC3EFE8E5B8F5C900034E0FCA3E0FDEFCB
:105CCE002DFDEE3CFC8C5B8D5C123DC69000E4E03D
:105CDE00B40263123D17900117E0D39406401BAE39
:105CEE002CAF2D900115E01273A274C88E048F058F
:105CFE00FF1273928C5B8D5C8006852C5B852D5C10
:105D0E00AE5BAF5C745E1273A274058E048F05FFDA
:105D1E00127392AE59AF5AED2FFFEC3EFE8E5B8F93
:105D2E005C900034E0FCA3E0FDEF2DFDEE3CFC8C1E
:105D3E005B8D5C123DC68009123CD8123D78123D37
:105D4E008E8024123CD8123D78123D8EA203B340B1
:105D5E0006123DA4123DC69000E4E0B40209123DC5
:105D6E0017123DA4123DC6C20CD20DA20DB3B350F4
:105D7E0008900041E0655E600302607AA202B350B3
:105D8E0006A201B3B340030260769000C6E0B404ED
:105D9E000280030260529008E8E0B402028003021F
:105DAE006047A21CB35003025F00123CD89001174B
:105DBE00E0D39401401F900014E0FEA3E0FF900199
:105DCE0010E01273A274C88E048F05FF1273928CAA
:105DDE005B8D5C800A900014E0F55BA3E0F55CAE91
:105DEE005BAF5C745E1273A274058E048F05FF1296
:105DFE007392AE59AF5AED2FFFEC3EFE8E5B8F5C69
:105E0E00900034E0FCA3E0FDEF2DFDEE3CFC8C5B3E
:105E1E008D5C123D83A203B3406B123D17900117A8
:105E2E00E0D39401401F900014E0FEA3E0FF900128
:105E3E0010E01273A274C88E048F05FF1273928C39
:105E4E005B8D5C800A900014E0F55BA3E0F55CAE20
:105E5E005BAF5C745E1273A274058E048F05FF1225
:105E6E007392AE59AF5AED2FFFEC3EFE8E5B8F5CF8
:105E7E00900034E0FCA3E0FDEF2DFDEE3CFC8C5BCE
:105E8E008D5C123DB59000E4E0B40263123D1790B4
:105E9E000117E0D39405401BAE2CAF2D900114E0FA
:105EAE001273A274C88E048F05FF1273928C5B8DD1
:105EBE005C8006852C5B852D5CAE5BAF5C745E12E0
:105ECE0073A274058E048F05FF127392AE59AF5AEA
:105EDE00ED2FFFEC3EFE8E5B8F5C900034E0FCA35A
:105EEE00E0FDEF2DFDEE3CFC8C5B8D5C123DB502B2
:105EFE006045123CD8900117E0D39403401F9000E8
:105F0E0014E0FEA3E0FF900112E01273A274C88E9B
:105F1E00048F05FF1273928C5B8D5C800A900014C7
:105F2E00E0F55BA3E0F55CAE5BAF5C745E1273A252
:105F3E0074058E048F05FF127392AE59AF5AED2F72
:105F4E00FFEC3EFE8E5B8F5C900034E0FCA3E0FD28
:105F5E00EF2DFDEE3CFC8C5B8D5C123D99A203B3E4
:105F6E00406B123D17900117E0D39403401F900031
:105F7E0014E0FEA3E0FF900112E01273A274C88E2B
:105F8E00048F05FF1273928C5B8D5C800A90001457
:105F9E00E0F55BA3E0F55CAE5BAF5C745E1273A2E2
:105FAE0074058E048F05FF127392AE59AF5AED2F02
:105FBE00FFEC3EFE8E5B8F5C900034E0FCA3E0FDB8
:105FCE00EF2DFDEE3CFC8C5B8D5C123DDB9000E416
:105FDE00E0B40263123D17900117E0D39407401B03
:105FEE00AE2CAF2D900116E01273A274C88E048FE2
:105FFE0005FF1273928C5B8D5C8006852C5B852D64
:10600E005CAE5BAF5C745E1273A274058E048F057A
:10601E00FF127392AE59AF5AED2FFFEC3EFE8E5B20
:10602E008F5C900034E0FCA3E0FDEF2DFDEE3CFC18
:10603E008C5B8D5C123DDB8009123CD8123D8312C5
:10604E003D998024123CD8123D83123D99A203B390
:10605E004006123DB5123DDB9000E4E0B402091299
:10606E003D17123DB5123DDBD20CC20DE570906CA2
:09607E0060F82828739000EBE0A3
:036C60000260834C
:10608700906CCFF82828731225CF80121225CF8065
:0E6097000D12265980081227058003122705D6
:0F6CCF0002608E02609302609802609D0260A2D4
:1060A5007570010264DD12283112294875700202EB
:1060B50064DD122CC8A204B340139000D0E075F043
:1060C5001DA4FFAEF0900010EEF0A3EFF090087E57
:1060D500E0FEA3E0FF740A1273A290000AE0FCA39D
:1060E500E0FD74098F02FF1273928D078C038E04F5
:1060F5008A058B06127290900882EEF0A3EFF0905D
:1061050000D4E0B401087478BE00059F4002800DFC
:106115007478900882F8E4F0E8A3F0801B90088278
:10612500E0FEA3E0FF74F0BE00039F500B74F090F7
:106135000882F8E4F0E8A3F0E536700375360190BF
:106145000882E0FEA3E0FFE5362FFF50010E900820
:1061550082EEF0A3EFF0757003A22E401590004A71
:01616500E059
:066C63000260AB0260B705
:10616600906CDEF8282873800875700A80037570B5
:016176000B1D
:096CDE0002616D02616F02617434
:106177000264DD9006C5E060077401F508122DF68C
:10618700A230B3401675E70090077CE0B42A06E515
:10619700B54402F5B575E7100262439000B9E0D344
:1061A7009402404590008DE02403A851B80004955F
:1061B70052500990008FE0D395615002800ED202B1
:1061C700A22640067408900049F0D22690008DE080
:1061D700A851B80005D39552500B90008FE02403C7
:1061E700C395615002C202805390008DE02403A83A
:1061F70051B8000495525010E55FC395605009905F
:10620700008FE0D395615002800ED202A22640068D
:106217007408900049F0D22690008DE0A851B8008C
:1062270005D395525014E560240FC3955F400B903A
:10623700008FE02403C395615002C202A20240020C
:10624700C226A230B35005A202B34002801375E7FD
:106257000090077CE0B42A06E5B554FDF5B575E76F
:10626700109000D3E07007E56AC3941440028002DF
:10627700D2029000C8E0B40102D202A20240057522
:106287007004800A757010900016E4F0A3F00264A1
:05629700DD9000B9E0FC
:066C690002617A0262984C
:10629C00906CE7F828287312135A801212135A8044
:0E62AC000D12150D80081215C480031215C4C2
:0F6CE7000262A30262A80262AD0262B20262B749
:1062BA009006C9E060077402F508122DF67570059C
:1062CA000264DD12171D7570069006CDE060077432
:1062DA0003F508122DF69006D1E060077404F5085C
:1062EA00122DF60264DD900044E06006A204B3B306
:1062FA004002800DE55ED394065006900044E014F7
:10630A00F01219A67570079006D5E060077405F5B6
:10631A0008122DF69006D9E060077406F508122DCA
:10632A00F60264DD900106E0B402031212CB121EDB
:10633A000E7570089006DDE060077407F508122DE7
:10634A00F69006E1E060077408F508122DF602647B
:10635A00DD121EF07570090264DD1222C8A20CB3A8
:10636A005005A20DB340028004D20CD20D757010F4
:10637A009006E5E060077409F508122DF69006E923
:10638A00E06007740AF508122DF60264DD90003801
:10639A00E0C39446500AC296C2A07446900038F0F0
:1063AA00900042E0B4011DE536241EF536900882BD
:1063BA00E0FEA3E0FF741E2FFF50010E900882EE4C
:1063CA00F0A3EFF085365A75590090003EE0F57358
:1063DA00123F95E55C900038F0900004E559F0A36F
:1063EA00E55AF0E573900039F0C20F900882E0F5A3
:1063FA0059A3E0F55A90003EE0F573123F95E55C2B
:10640A00900036F0900000E559F0A3E55AF0E573E4
:10641A00900037F0A2009210900042E06002B210A1
:10642A00C20E7570030264DD90003CE0C3944650CE
:10643A00139000D4E0B40102C296C295C297744682
:10644A0090003CF0900043E0B4011DE536241EF5AF
:10645A0036900882E0FEA3E0FF741E2FFF50010E63
:10646A00900882EEF0A3EFF085365A755900900035
:10647A003FE0F573123F95E55C90003CF090000612
:10648A00E559F0A3E55AF0E57390003DF0C2129089
:10649A000882E0F559A3E0F55A90003FE0F573123F
:1064AA003F95E55C90003AF0900002E559F0A3E5CB
:1064BA005AF0E57390003BF0A2009213900043E07B
:1064CA006002B213C21175700380088006800480CE
:0364DA000280003D
:106C6F000262CD0262F002632E02635B0263640272
:106C7F0063970264320264D50264D70264D9026456
:046C8F00DB0264DDE3
:1064DD00900036E0B55E0280030265A4A20E405C1A
:1064ED00900000E0FEA3E0FFEF4E602EAC55AD56E0
:1064FD007405FF1273928D068C07900000E0FCA3CB
:10650D00E0FDCFCECF12000374068E048F05FF126F
:10651D007392900000ECF0A3EDF0900037E0601A5C
:10652D00900000E0FEA3E0FFAC55AD56EF2DFDEE63
:10653D003CFC900000ECF0A3EDF0D20EAE53AF5446
:10654D00900000E0FCA3E0FDEFC39DEE9C404812DF
:10655D004C139000D4E0906C93F82828738030D2BF
:10656D0096802CD2968028D296D2A08022A210405E
:10657D0010A224301901B34004D2A08002D296801B
:0F658D000EA224301901B34004D2968002D2A08E
:0F6C930002656A02656C02657002657402657ABB
:10659C00C20E74C8900036F0A20EB3B35007900030
:1065AC0036E0B55E028048124C139000D4E0906C3B
:1065BC00A2F82828738030D296802CD2968028D2CC
:1065CC0096D2A08022A2104010A224301901B34010
:1065DC0004D2A08002D296800EA224301901B340BE
:0765EC0004D2968002D2A048
:0F6CA2000265C10265C30265C70265CB0265D1F9
:1065F30074C8900036F0C20E900038E0B55E7FA2FA
:106603000F405C900004E0FEA3E0FFEF4E602EAC71
:1066130055AD567405FF1273928D068C07900004D6
:10662300E0FCA3E0FDCFCECF12000374068E048FEF
:1066330005FF127392900004ECF0A3EDF090003983
:10664300E0601A900004E0FEA3E0FFAC55AD56EF06
:106653002DFDEE3CFC900004ECF0A3EDF0D20FAE68
:1066630053AF54900004E0FCA3E0FDEFC39DEE9C08
:10667300400CC296C2A07446900038F0C20FA20F1D
:10668300B3B35007900038E0B55E02800CC296C2E7
:10669300A07446900038F0C20F90003AE0B55E0255
:1066A3008003026763A211405C900002E0FEA3E056
:1066B300FFEF4E602EAC55AD567405FF1273928DED
:1066C300068C07900002E0FCA3E0FDCFCECF1200C2
:1066D3000374068E048F05FF127392900002ECF090
:1066E300A3EDF090003BE0601A900002E0FEA3E00F
:1066F300FFAC55AD56EF2DFDEE3CFC900002ECF0E7
:10670300A3EDF0D211AE53AF54900002E0FCA3E02E
:10671300FDEFC39DEE9C4048124C139000D4E090D3
:106723006CB1F82828738030D296802CD2958028BB
:10673300D295D2978022A2134010A225301901B31B
:106743004004D2978002D295800EA225301901B35E
:086753004004D2958002D297A8
:0F6CB10002672902672B02672F026733026739D8
:10675B00C21174C890003AF0A211B3B35007900065
:10676B003AE0B55E028048124C139000D4E0906C76
:10677B00C0F82828738030D296802CD2958028D2EE
:10678B0095D2978022A2134010A225301901B34055
:10679B0004D2978002D295800EA225301901B34006
:0767AB0004D2958002D29791
:0F6CC00002678002678202678602678A02679016
:1067B20074C890003AF0C21190003CE0B55E0280CD
:1067C2000302684EA212405C900006E0FEA3E0FFC6
:1067D200EF4E602EAC55AD567405FF1273928D06C6
:1067E2008C07900006E0FCA3E0FDCFCECF120003A1
:1067F20074068E048F05FF127392900006ECF0A3CC
:10680200EDF090003DE0601A900006E0FEA3E0FF8C
:10681200AC55AD56EF2DFDEE3CFC900006ECF0A31E
:10682200EDF0D212AE53AF54900006E0FCA3E0FDAF
:10683200EFC39DEE9C40159000D4E0B40102C296D5
:10684200C295C297744690003CF0C212A212B3B332
:10685200500790003CE0B55E0280159000D4E0B491
:106862000102C296C295C297744690003CF0C212D1
:106872009000D6E0B4020280030269A6900069E0AB
:10688200D395665064900069E0F4042566FE90009A
:10689200D9E08E00F5F0E884FF7E008F73EFC39499
:1068A20010500CEF8573F0A4FDACF08D738003756E
:1068B20073FF900069E0D39573400B900069E0C3C9
:1068C2009573F57180037571009000F4E0D39571B2
:1068D20040069000F4E0F5719000F5E0C395715028
:1068E200069000F5E0F5718071900069E0C395664D
:1068F200FE9000D9E08E00F5F0E884FF7E008F73F1
:10690200EFC39410500CEF8573F0A4FDACF08D73BF
:1069120080037573FF85735A755900900069E025ED
:106922005AFFAE5950010E8E598F5A74FFBE00099C
:10693200D39F4005855A7180037571FF9000F4E082
:10694200D3957140069000F4E0F5719000F5E0C334
:10695200957150069000F5E0F571A204B3B3500DA5
:1069620090006AE0FE9000E1E0D39E500280147431
:1069720007900049F075E700E5B554BFF5B575E736
:1069820010802175A71075E700E5CDC39571400809
:10699200E5B554BFF5B58006E5B54440F5B575E7F4
:1069A2001075A7009000F1E0604E9000FBE0A85146
:1069B200B80004955250179000FAE0A851B8000EA2
:1069C200D3955240099000FCE0D3956140028015B6
:1069D20075A710E5CDC394BF4004C2A28002D2A223
:1069E20075A700801375A710E5CDC394404004C27B
:1069F200A28002D2A275A7009000F2E0604E900041
:106A0200FEE0A851B80004955250179000FDE0A88E
:106A120051B8000ED3955240099000FFE0D3956122
:106A22004002801575A710E5CDC394BF4004C2A1F2
:106A32008002D2A175A700801375A710E5CDC3947B
:106A4200404004C2A18002D2A175A700E56FC394A1
:106A520013501DE56F75F00284AFF07E00EF4E70AB
:106A620005123290800AA2EDB34005C2ED123290B7
:106A7200AE53AF547430C39F74759E400C9000683F
:106A8200E0C3945A4003026C06A209B340091247BC
:106A9200387406900049F0A20BB3500EE561D3940E
:106AA200334007E561C394CC40028041900106E087
:106AB200B4021412124490006DE075F05EA4FFAEB1
:106AC200F08E5B8F5C800F900082E075F05EA4FF19
:106AD200AEF08E5B8F5CE55C455B6011E5B5440111
:106AE200F5B5742B900067F0124B75D20B900068CD
:106AF200E0D394014007E561C3941A40028002C2C8
:106B02000B9006C5E060077401F508122DF6900699
:106B1200C9E060077402F508122DF69006CDE06018
:106B2200077403F508122DF69006D1E0600774048D
:106B3200F508122DF69006D5E060077405F50812E7
:106B42002DF69006D9E060077406F508122DF6902E
:106B520006DDE060077407F508122DF69006E1E005
:106B620060077408F508122DF69006E5E0600774D8
:106B720009F508122DF69006E9E06007740AF50897
:106B8200122DF6900068E0C3945A5010E56FB413CA
:106B920009900068E004F0756F00803FE56FB41360
:106BA20003756F00C28E758D00758B00756400755C
:106BB2005401755300D28E900067E0C3944150088F
:106BC200900067E004F080067441900067F0900046
:106BD20067E0B44106E5B554FEF5B5900068E0D330
:106BE20094014007E56AC3944140028006740E9006
:106BF2000049F0900895E06006900103E060028091
:076C020003120B970250FB87
:106CF6000000010001400160018001A001C001E027
:106D060002000300039603B603D603F4040005004D
:106D16000512052405360548055A056C057E0590BD
:106D260005A805C005DE0600061406280646066EFA
:106D360006AE05CF06EE00FF013F015F017F019F12
:106D460001BF01DF01FF02FF039503B503D503F37E
:106D560003FF04FF05110523053505470559056B96
:106D6600057D058F05A705BF05CE05F10613062788
:106D76000645066D06AD06ED05DD06FF0FAA0FA555
:106D86000F9F0F9A0F940F8D0F870F800F780F713B
:106D96000F680F600F570F4E0F450F3B0F300F2533
:106DA6000F1A0F0E0F020EF50EE80EDB0ECC0EBEFE
:106DB6000EAE0E9F0E8E0E7D0E6C0E5A0E470E34C4
:106DC6000E200E0C0DF70DE20DCB0DB50D9D0D85AC
:106DD6000D6D0D540D3A0D200D050CE90CCE0CB1C0
:106DE6000C940C760C580C3A0C1B0BFB0BDB0BBBF8
:106DF6000B9A0B790B570B350B130AF10ACE0AAB1C
:106E06000A870A640A400A1C09F809D409B0098CE1
:106E160009670943091F08FB08D608B2088E086AE5
:106E26000846082307FF07DC07B9079607730751CB
:106E3600072F070D06EC06CA06AA06890669064943
:106E4600062A060A05EC05CD05B005920575055816
:106E5600053C0520050504EA04CF04B5049C04821C
:106E66000469045104390422040B03F403DE03C845
:106E760003B2039D038903750361034D033B032896
:106E86000316030402F202E102D102C002B002A01C
:106E9600029102820273026502570249023C022FE6
:106EA60002220216020901FD01F201E601DB01D010
:106EB60001C601BB01B101A7019D0194018B0182AD
:106EC60001790170016801600158015001480141D2
:106ED60001390132012B0125011E01180111010B97
:106EE600010500FF00FA0FA60FA00F990F920F8B56
:106EF6000F840F7C0F740F6B0F620F580F4E0F43EA
:106F06000F380F2C0F1F0F120F050EF70EE80ED8B5
:106F16000EC80EB70EA50E930E800E6C0E580E42BE
:106F26000E2C0E150DFD0DE40DCB0DB10D950D7945
:106F36000D5D0D3F0D200D010CE10CC00C9E0C7C6F
:106F46000C590C350C100BEA0BC40B9E0B760B4F31
:106F56000B260AFD0AD40AAA0A800A550A2A09FF3C
:106F660009D409A8097C0950092508F908CD08A102
:106F76000875084A081E07F307C8079D07730749DF
:106F8600072006F706CE06A6067E06570630060A30
:106F960005E405BF059B057705540532051004EF8A
:106FA60004CE04AE048F047104530435041903FDA2
:106FB60003E203C703AD0394037B0363034B03346C
:106FC600031E030802F302DE02CA02B602A30291FE
:106FD600027F026D025C024C023C022C021D020E74
:106FE600020001F201E401D701CA01BE01B101A606
:106FF600019A018F0185017A01700166015D0153D5
:10700600014A014101390131012901210119011208
:10701600010B010400FD00F700F000EA00E400DEC9
:1070260000D900D300CE00C900C400BF00BA00B525
:1070360000B100AD00A800A400A0009C0099009536
:107046000091008E008A008700840081007E007B0C
:10009E0075B50075840175A70075FFA075EF069004
:1000AE000045E4F075C91075A70F75A1C775A700B7
:1000BE0075D90075CE0C75A70F75F1FE75F2FF752B
:1000CE00F30775F47875A4BA75A5FF75A60775AE16
:1000DE000075AFFF75D48175D5FF75D6FF75D7FF47
:1000EE0075A70075A20175A14775F8092275E60876
:1000FE0075E71075BC0175BE0475BD6C75BE0775D0
:10010E00BDA075BE0875BD0175BC0075BB1875BC6C
:10011E002075BA0875E88075D11375A70F75E105BE
:10012E0075E20075C7401247387597007597807451
:10013E000A1273827597C0E5975420700280F87585
:10014E008F0275A700D2AF75980075A90C75A70F11
:10015E0075AB4375ADFB75AC1E75A71075C91875DB
:10016E00CA0075CB0075C80475A700758912758E07
:10017E0004758C00758A00C2A9D28C758D00758BA2
:10018E0000D2ABD28E75B62075D944C2992290009A
:10019E0080E0900894F090008BE0900895F090002D
:1001AE008CE0900896F09000ABE0900897F09000ED
:1001BE00B8E0900898F09000C6E0900899F0900092
:1001CE00D4E090089AF09000D6E090089BF0900052
:1001DE00E4E090089CF09000F1E090089DF0900013
:1001EE00F2E090089EF0900104E090089FF09001DC
:1001FE001CE09008A1F090016AE09008A2F0900136
:10020E006BE09008A3F090016CE09008A4F09001D0
:10021E0003E09008A5F09000EDE09008A6F09000A5
:10022E00A4E09008A7F09000A5E09008A8F0900038
:10023E009FE09008A9F09000A0E09008AAF090012D
:10024E0009E09008ABF090010AE09008ACF0900144
:10025E000BE09008ADF090010CE09008AEF090012C
:10026E000DE09008AFF09006C4E09008B0F0900654
:10027E00C8E09008B1F09006CCE09008B2F090067D
:10028E00D0E09008B3F09006D4E09008B4F0900659
:10029E00D8E09008B5F09006DCE09008B6F0900635
:1002AE00E0E09008B7F09006E4E09008B8F0900611
:1002BE00E8E09008B9F090076CE09008BAF090076B
:1002CE006DE09008BBF090076EE09008BCF09007D0
:1002DE006FE09008BDF0900770E09008BEF09007B8
:1002EE0071E09008BFF0900772E09008C0F09007A0
:1002FE0073E09008C1F0900774E09008C2F0900788
:10030E0075E09008C3F0900776E09008C4F090076F
:10031E0077E09008C5F0900778E09008C6F0900757
:10032E0079E09008C7F090077AE09008C8F090073F
:10033E007BE09008C9F090077CE09008CAF090012D
:10034E000EE09008CBF090010FE09008CCF09001F9
:10035E0010E09008CDF0900111E09008CEF09001E1
:10036E0012E09008CFF0900113E09008D0F09001C9
:10037E0014E09008D1F0900115E09008D2F09001B1
:10038E0016E09008D3F0900117E09008D4F0229078
:10039E000894E0900080F0900895E090008BF0902B
:1003AE000896E090008CF0900897E09000ABF090EB
:1003BE000898E09000B8F0900899E09000C6F09090
:1003CE00089AE09000D4F090089BE09000D6F09050
:1003DE00089CE09000E4F090089DE09000F1F09011
:1003EE00089EE09000F2F090089FE0900104F090DB
:1003FE0008A1E090011CF09008A5E0900103F09098
:10040E0008A6E09000EDF09008A7E09000A4F09010
:10041E0008A8E09000A5F09008A9E090009FF09049
:10042E0008AAE09000A0F09008ABE0900109F090CF
:10043E0008ACE090010AF09008ADE090010BF0904E
:10044E0008AEE090010CF09008AFE090010DF09036
:10045E0008B0E09006C4F09008B1E09006C8F090A5
:10046E0008B2E09006CCF09008B3E09006D0F09081
:10047E0008B4E09006D4F09008B5E09006D8F0905D
:10048E0008B6E09006DCF09008B7E09006E0F09039
:10049E0008B8E09006E4F09008B9E09006E8F09015
:1004AE0008BAE090076CF09008BBE090076DF090F2
:1004BE0008BCE090076EF09008BDE090076FF090DA
:1004CE0008BEE0900770F09008BFE0900771F090C2
:1004DE0008C0E0900772F09008C1E0900773F090AA
:1004EE0008C2E0900774F09008C3E0900775F09092
:1004FE0008C4E0900776F09008C5E0900777F0907A
:10050E0008C6E0900778F09008C7E0900779F09061
:10051E0008C8E090077AF09008C9E090077BF09049
:10052E0008CAE090077CF09008CBE090010EF090A6
:10053E0008CCE090010FF09008CDE0900110F09003
:10054E0008CEE0900111F09008CFE0900112F090EB
:10055E0008D0E0900113F09008D1E0900114F090D3
:10056E0008D2E0900115F09008D3E0900116F090BB
:10057E0008D4E0900117F02275470090088CE4F043
:10058E00A3F0753100753000754D00754E00C22A0E
:10059E00D22B900895E06002D22074FE90088EF85F
:1005AE00E4F0E8A3F074FE900892F8E4F0E8A3F00B
:1005BE0074FE900890F8E4F0E8A3F0745A9008E600
:1005CE00F0745A9008E7F0D22CC228C22EC22DC267
:1005DE0029C230C23622750B00750A00AE0AAF0B67
:1005EE00AC08AD09EDC39FEC9E401674FF127382EA
:1005FE0075CF01780B740126F6500418E436F650C8
:10060E00DB22C2AF75D904758F0375B7A575B7F127
:10061E0090F800E4F0758F0175B7A575B7F1E52771
:10062E0090F800F075B7A575B7F190F801E4F07584
:10063E00B7A575B7F19008DAE090F802F075B7A596
:10064E0075B7F19008DEE090F803F075B7A575B7B1
:10065E00F19008DBE090F804F075B7A575B7F1904E
:10066E0008DCE090F805F075B7A575B7F19008DDD8
:10067E00E090F806F075B7A575B7F19008DFE09039
:10068E00F807F0758F0075D944D2AF22900045E07F
:10069E00B4AB61C2AF75D90475B62275F522758FEC
:1006AE000375B7A575B7F1740090F600F0758F015C
:1006BE00755A00755900AE59AF5A7445BE00279F42
:1006CE00402475B7A575B7F1900894120048E0FC68
:1006DE0090F600120048ECF0785A740126F6500499
:1006EE0018E436F650D0758F0075F51175B6207575
:1006FE00D944D2AF22C2AF75F52275D904755A000E
:10070E00755900AE59AF5A7445BE00229F401F90D6
:10071E00F600120048E493FC900894120048ECF0A6
:10072E00785A740126F6500418E436F650D575D969
:10073E004475F511D2AF22900045E0B4AA028003B1
:10074E00020882C2AF75D90475B62275F522758F6F
:10075E000375B7A575B7F1740090F400F075B7A5E1
:10076E0075B7F1740090F200F075B7A575B7F17416
:10077E000090F000F075B7A575B7F1740090EE001B
:10078E00F0758F01755A00755900AE59AF5A74FF46
:10079E00C39F74019E402475B7A575B7F190007E76
:1007AE00120048E0FC90F400120048ECF0785A7405
:1007BE000126F6500418E436F650CF755A007559D6
:1007CE0000AE59AF5A74FFC39F74019E402475B793
:1007DE00A575B7F190027E120048E0FC90F200126F
:1007EE000048ECF0785A740126F6500418E436F6F8
:1007FE0050CF755A00755900AE59AF5A74FFC39F4A
:10080E0074019E402475B7A575B7F190047E120051
:10081E0048E0FC90F000120048ECF0785A74012683
:10082E00F6500418E436F650CF755A00755900AEDE
:10083E0059AF5A74FFC39F74019E402475B7A575B6
:10084E00B7F190067E120048E0FC90EE00120048D0
:10085E00ECF0785A740126F6500418E436F650CFB0
:10086E00758F0075F51175B62075D944D2AF743AEF
:10087E0090077EF022900045E0B4AA0280030209A0
:10088E00C0C2AF75D90475B62275F522758F037582
:10089E00B7A575B7F1740090EC00F075B7A575B7F4
:1008AE00F1740090EA00F075B7A575B7F174009079
:1008BE00E800F075B7A575B7F1740090E600F07515
:1008CE008F01755A00755900AE59AF5A74FFC39F08
:1008DE0074019E402475B7A575B7F190007E120085
:1008EE0048E0FC90EC00120048ECF0785A740126B7
:1008FE00F6500418E436F650CF755A00755900AE0E
:10090E0059AF5A74FFC39F74019E402475B7A575E5
:10091E00B7F190027E120048E0FC90EA0012004807
:10092E00ECF0785A740126F6500418E436F650CFDF
:10093E00755A00755900AE59AF5A74FFC39F7401B2
:10094E009E402475B7A575B7F190047E120048E05D
:10095E00FC90E800120048ECF0785A740126F6502C
:10096E000418E436F650CF755A00755900AE59AFDB
:10097E005A74FFC39F74019E402475B7A575B7F1D5
:10098E0090067E120048E0FC90E600120048ECF063
:10099E00785A740126F6500418E436F650CF758F47
:1009AE000075F51175B62075D944D2AF743A90071B
:1009BE007EF022C2AF75D90475F522755A007559AD
:1009CE0000AE59AF5A74FFC39F74019E401F90F43E
:1009DE0000120048E493FC90007E120048ECF07880
:1009EE005A740126F6500418E436F650D4755A009F
:1009FE00755900AE59AF5A74FFC39F74019E401FC4
:100A0E0090F200120048E493FC90027E120048EC33
:100A1E00F0785A740126F6500418E436F650D47560
:100A2E005A00755900AE59AF5A74FFC39F74019E98
:100A3E00401F90F000120048E493FC90047E1200D8
:100A4E0048ECF0785A740126F6500418E436F65045
:100A5E00D4755A00755900AE59AF5A74FFC39F74BE
:100A6E00019E401F90EE00120048E493FC90067E1B
:100A7E00120048ECF0785A740126F6500418E43649
:100A8E00F650D475F51175D944D2AF74019000C7E4
:100A9E00F0743A90077EF09008ED7401F022C2AF28
:100AAE0075D90475F522755A00755900AE59AF5AAD
:100ABE0074FFC39F74019E401F90EC00120048E427
:100ACE0093FC90007E120048ECF0785A740126F6E2
:100ADE00500418E436F650D4755A00755900AE59C4
:100AEE00AF5A74FFC39F74019E401F90EA0012001C
:100AFE0048E493FC90027E120048ECF0785A7401A0
:100B0E0026F6500418E436F650D4755A007559007E
:100B1E00AE59AF5A74FFC39F74019E401F90E800F8
:100B2E00120048E493FC90047E120048ECF0785AD0
:100B3E00740126F6500418E436F650D4755A007532
:100B4E005900AE59AF5A74FFC39F74019E401F9057
:100B5E00E600120048E493FC90067E120048ECF08A
:100B6E00785A740126F6500418E436F650D475F50A
:100B7E001175D944D2AF74029000C7F0743A900741
:100B8E007EF074029008EDF02274019000C7F09090
:100B9E000895E0903C1EF828287380188016A2A3B2
:100BAE00400674029000C7F0800AA2A440067402A8
:040BBE009000C7F0EC
:0C3C1E00020BA8020BAA020BAC020BB8B0
:100BC2009000C7E0B40105A234B34002801AD234C7
:100BD2001247381209C174019000C7F012039D1226
:100BE2003EB7741B900049F09000C7E0B40206A221
:100BF20034B3B34002801AC234124738120AAC74BA
:100C0200029000C7F012039D123EB7741B90004978
:100C1200F022E54E64046006E59964FF60028031CB
:100C2200A22A4004D22A8027E54E600874E6254EA7
:100C3200900049F0E54D600874F0254D900049F0B0
:100C4200E54EB4010280FE754E00754D00C22A8049
:100C520002C22AE54E903C2AF8282873754E00E518
:100C620099B4FF03754D01E599B4FE03754D02E594
:100C720099B4FD03754D03E599B4FC03754D04E584
:100C820099B4FA03754D05E599B4FB06754E011248
:100C92004738E599B4F906754E04124738E599B418
:100CA200F733124738C29C74AB900045F012069A93
:100CB20074AA900045F09008EDE0B40105120745D2
:100CC2008003120883900045E4F0D29C754E0075B3
:100CD2004D007599F7E599D394E54007E599C394DA
:100CE200F04002801685994F754E027E017F00E525
:100CF2004FC394E61273A28E328F3390088CE4F0C5
:100D0200A3F0E599D394C24007E599C394E6400263
:100D1200802885994F754E0374E5C3954FF5337559
:100D22003200AE32AF33906CF6127371E493F87402
:100D3200019390088CC8F0A3C8F0D2990210A29037
:100D420008A1E0700AA221B35005A222B34002809A
:100D52005C90088CE0FEA3E0FF74FFBE00039F508E
:100D620009EFC39446EE9406402B90088CE0FEA354
:100D7200E0FFEFD3946DEE94064009EFC394EEEEDC
:100D82009406401190088CE0FEA3E0FFEFD394FF9D
:100D9200EE9406401390088CE0FEA3E0FF90007EE4
:100DA200120048E599F08003859974801190088CAF
:100DB200E0FEA3E0FF90007E120048E599F0900863
:100DC2008C1273B090088CE0FEA3E0FFEFB4010632
:100DD200EEB407028003020E9B90077EE0B43C0251
:100DE2008003020E9BA221B35005A222B3400280CF
:100DF20055C29C12039D90008BE09008ECF01240CB
:100E02001B90016AE09008A2F090016BE09008A3A9
:100E1200F090016CE09008A4F074AB900045F012E1
:100E2200069A74AA900045F09008EDE0B40105120C
:100E3200074580031208839008EDE09000C7F09008
:100E42000045E4F08048C29C12019C74009008A204
:100E5200F074009008A3F074009008A4F090008B46
:100E6200E09008ECF012401B74AB900045F01206C3
:100E72009A74AA900045F0120745120883D29C7515
:100E820099FB7464F5097508001205E480FED29C92
:100E9200754E00754D007599FB0210A290088CE00A
:100EA200FEA3E0FFEF4E7006859931753000900881
:100EB2008CE0FEA3E0FF74016F4E701BAC30AD31CD
:100EC200AA32AB33ED2BFBEC3AFA8A068B07900081
:100ED2007E120048E599F090088C1273B090088C4D
:100EE200E0FEA3E0FF74026F4E7021AC30AD3174AE
:100EF200566D4C7006E54F64E66002800312473877
:100F020012401B854F99754E00754D000210A2903C
:100F1200088CE0FEA3E0FF90007E120048E599F005
:100F220090088C1273B090088CE0FEA3E0FFAC3204
:100F3200AD338F028E038C068D07906D3C12737158
:100F4200E493F9740193FEEAD39EEB994009854F2D
:100F520099754E00754D000210A290088CE0FEA318
:100F6200E0FF90007E120048E599F090088C127321
:100F7200B090088CE0FEA3E0FFEFB40006EEB401EF
:100F82000280030210A290005BE0D394C7400B9052
:100F9200005BE0C394C8F550801A90005BE0D394E4
:100FA20063400B90005BE0C39464F55080069000B0
:100FB2005BE0F550E55075F002A4FFAEF08F73EFE1
:100FC20090007E1273D3EFFCE0FDEC90008112736F
:100FD200D3EDFCE0FDEC2DB5500280030210930F1F
:100FE200EF90007E1273D3E573FFE0FCEF90008276
:100FF2001273D3ECFFE0FCEFC39CB55002800302F6
:101002001093E5739000801273D3E573FFE0FCEF59
:101012009000831273D3ECFFE0FCEF2CB55072E525
:10102200739000841273D3E0C395509008DAF0E510
:10103200739000851273D3E0C395509008DBF0E5FE
:10104200739000881273D3E0C395509008DCF0E5EA
:10105200739000891273D3E0C395509008DDF0E5D8
:101062007390008A1273D3E0C395509008DEF0E5C6
:101072007390008B1273D3E0C395509008DFF01287
:1010820006107599F97464F5097508001205E48073
:10109200FE7599FF7464F5097508001205E480FE77
:0F3C2A00020C5E020D41020E9E020F11020F5C92
:1010A20022E54D903C39F828287302118790088C6C
:1010B200E0FEA3E0FF90004B120048E0F599900893
:1010C2008C1273B090088CE0FEA3E0FF741C6F4E8C
:1010D2007003754D00021187856E99021187900881
:1010E2008CE0FEA3E0FF90007E120048E0F599EF4D
:1010F200B40107EEB40703754D0090088C1273B06B
:0711020002118790088DE047
:0F3C39000210AC0210AF0210DA0210E002110507
:10110900903CABF82828738552998067855F998050
:1011190062856199805D8565998058856799805355
:10112900856899804E8569998049856A9980449036
:101139000017E0F599803CA22BB340077599FAC2D4
:101149002B8017A220B3400575990F800B90004999
:10115900E0F599900049E4F0C2208017856B9980E9
:1011690012856699800D856C9980087599FC8003B4
:03117900754D00B1
:103CAB0002111002111502111A02111F0211240226
:103CBB00112902112E021133021138021140021187
:0D3CCB006502116A02116F02117402117975
:0B117C0090088C1273B08003123F1229
:033C4800021184E2
:1011870022E537255AFFAE5950010E90007E120016
:1011970048E0F538E537255AFFAE5950010E0FBF25
:1011A70000010E90007E120048E0F539853F3BE5CF
:1011B70038B539058538378041E539D39538401D2D
:1011C700E539C39538853AF0A4FFAEF0E53B8E04C8
:1011D7008F05FF127392ED2538F537801DE538C36B
:1011E7009539853AF0A4FFAEF0E53B8E048F05FFF5
:1011F700127392EDF4042538F53722E539D3953883
:10120700401DE539C39538853AF0A4FFAEF0E53BBC
:101217008E048F05FF127392ED2538F537801DE593
:1012270038C39539853AF0A4FFAEF0E53B8E048FBD
:1012370005FF127392EDF4042538F53722900084E8
:10124700E0B4017FE56775F00A84FF7E008F37E51C
:101257006775F00A84ADF07C008D3A753F0A7559C1
:1012670005755A24E537C394115005121188800675
:101277009005B3E0F537E537C394F05008E53790AC
:10128700006DF0800674EF90006DF0E56775F00A69
:1012970084FF7E008F37E56775F00A84ADF07C0028
:1012A7008D3A753F0A755905755A5AE537C3941132
:1012B700500512118880069005E9E0F537E537906B
:1012C7000044F022900084E0B40102800302135925
:1012D700E56775F00A84FF7E008F37E56775F00ACA
:1012E70084ADF07C008D3A753F0A755905755A36FD
:1012F700E537C39411500512118880069005C5E0A3
:10130700F537E537C394F0500585374B8003754BA8
:10131700EFE56775F00A84FF7E008F37E56775F0A4
:101327000A84ADF07C008D3A753F0A755905755AE8
:1013370048E537C39411500512118880069005D7E8
:10134700E0F537E537C394F0500585374C800375D2
:101357004CEF22E55F75F00484FF7E008F37E55F71
:1013670075F00484ADF07C008D3A753F0475590122
:10137700755A00E537C3943F5005121188800690CF
:1013870001BDE0F537E537900886F8E4F0E8A3F00B
:10139700900048E075F020A4FFAEF09000CFE08EFB
:1013A700048F05FF1273928D379000B7E0D3955FD6
:1013B70050030214659000DBE0D3955F4010ED9079
:1013C70001BE1273D3E0F52B752A00021462900058
:1013D700A6E0D3955F4043E5379001BE1273D3E093
:1013E700F538E5379001DE1273D3E0F5399000DB6D
:1013F700E0F404255FF53A9000A6E0FE9000DBE0FC
:10140700F4042EF53BE538B53905853837800312E6
:10141700120285372B752A008041E5379001DE12CD
:1014270073D3E0F538E5379001FE1273D3E0F53951
:101437009000A6E0F404255FF53A9000B7E0FE902F
:1014470000A6E0F4042EF53BE538B53905853837B5
:10145700800312120285372B752A0002150C9000A3
:10146700DEE0D3955F5011E53790023E1273D3E06B
:10147700F52B752A0002150C9000A7E0D3955F5055
:1014870043E53790021E1273D3E0F538E537900233
:101497003E1273D3E0F5399000A7E0F404255FF519
:1014A7003A9000DEE0FE9000A7E0F4042EF53BE55D
:1014B70038B53905853837800312120285372B7501
:1014C7002A008041E5379001FE1273D3E0F538E535
:1014D7003790021E1273D3E0F5399000B7E0F40499
:1014E700255FF53A9000A7E0FE9000B7E0F4042EE0
:1014F700F53BE538B5390585383780031212028583
:10150700372B752A00229000EFE0F53C753F1175E7
:101517005902755A00AE51AF52E53C75F00FA4FD64
:10152700ACF0EDD39FEC9E4021E53C8E048F05FF88
:10153700127392ED75F010A4FFAEF0E55F75F01130
:1015470084FD7C00ED2FF53D800EE55F75F011847D
:10155700FF7E00EF24F0F53D853D37E55F75F0111F
:1015670084AFF07E008F3A12118885373EAE51AFB7
:10157700529000EFE075F00FA4FDACF0EDD39FECB7
:101587009E4028755902755A10853D371211888576
:101597003E38853739AE51AF52E53C8E048F05FF93
:1015A7001273BD8D3A853C3B121202E537900886CF
:1015B700F8E4F0E8A3F0752B64752A00229000EF99
:1015C700E0F53C753F11755902755A00AE51AF529F
:1015D700E53C75F00FA4FDACF0EDD39FEC9E4021E8
:1015E700E53C8E048F05FF127392ED75F010A4FF92
:1015F700AEF0E56175F01184FD7C00ED2FF53D80BF
:101607000EE56175F01184FF7E00EF24F0F53D854E
:101617003D37E56175F01184AFF07E008F3A121106
:101627008885373EAE51AF529000EFE075F00FA4BA
:10163700FDACF0EDD39FEC9E4028755902755A100A
:10164700853D37121188853E38853739AE51AF52FF
:10165700E53C8E048F05FF1273BD8D3A853C3B1226
:101667001202E537900886F8E4F0E8A3F0E56B602E
:1016770017E56BC394FE50109000E3E0B4020990A5
:1016870000D1E0D3940B5002801F900886E0FEA3A0
:10169700E0FFE56B1273A274E78E048F05FF1273E8
:1016A70092900886ECF0A3EDF09000B9E0B4045FE7
:1016B700E55F75F00484FF7E008F37E55F75F00402
:1016C70084ADF07C008D3A753F04755901755A0059
:1016D700E537C3943F500512118880069001BDE09D
:1016E700F537900886E0FEA3E0FFE5371273A27492
:1016F700328E048F05FF127392900886E0FEA3E0F6
:10170700FFEF2DFDEE3CFC900886ECF0A3EDF075A5
:101717002B64752A0022900084E0B40146E56775C2
:10172700F00A84FF7E008F37E56775F00A84ADF015
:101737007C008D3A753F0A755905755A00E537C320
:1017470094115005121188800690058FE0F537AE89
:101757002AAF2BE5372FFF50010E74641273E58E05
:101767002A8F2B900085E0B40146E56875F00A845E
:10177700FF7E008F37E56875F00A84ADF07C008D39
:101787003A753F0A755905755A6CE537C394115078
:101797000512118880069005FBE0F537AE2AAF2BBE
:1017A700E5372FFF50010E74641273E58E2A8F2BD5
:1017B700900094E0B40249E56AC3944175F005844A
:1017C700FF7E008F37E56A75F00584ADF07C008DEC
:1017D7003A753F05755906755A00E537C394135096
:1017E700051211888006900691E0F537AE2AAF2BD7
:1017F700E5372FFF50010E74641273E58E2A8F2B85
:101807009000D6E0B4020280030218BCE55F75F0D1
:101817001584FF7E008F37E55F75F01584ADF07C8A
:10182700008D3A753F15755903755AF4E537C3941A
:101837000B5005121188800690047DE0F537E537D7
:1018470075F0FFA4FFAEF09000D7E08E048F05FF80
:10185700127392ED900069F0E56675F078A4FFAE1B
:10186700F074FF8E048F05FF1273928C598D5A7492
:10187700028C068D071200398F37AC59AD5A7404A4
:10188700FF1273BD8D3A753F04755906755A28E5E1
:1018970037C3941D500512118880069006C3E0F5E2
:1018A70037AE2AAF2BE5372FFF50010E7464127342
:1018B700E58E2A8F2B900083E0B4025DE56175F019
:1018C70064A4FFAEF074081200398E5B8F5C740558
:1018D7008E048F05FF1273928D37AE5BAF5C740574
:1018E7008E048F05FF1273BD8D3A753F0575590537
:1018F700755ADEE537C39413500512118880069098
:10190700066FE0F537AE2AAF2BE5372FFF50010EF4
:1019170074641273E58E2A8F2B9000C5E0707F9058
:101927000048E075F00A84FF7E008F37900048E09A
:1019370075F00A84ADF07C008D3A753F0A7559053C
:10194700755AC0E537C3940E50051211888006906A
:10195700064CE0F537E53790006EF09000E4E0B410
:10196700023C900048E075F00A84FF7E008F3790B4
:101977000048E075F00A84ADF07C008D3A753F0AA7
:10198700755905755ACFE537C3940E50051211885E
:10199700800690065BE0F537E53790006FF0229000
:1019A700008CE0B401179008E1E0252BFFAE2A5028
:1019B700010E9000E0E01273E58E2A8F2B90010450
:1019C700E0B40114900105E0A851B8000495525005
:1019D70007E55FC39560400280139000AEE0252BBA
:1019E700FFAE2A50010E8E2A8F2B021E0D90008CFF
:1019F700E0B40306A228B3B3400280509008EBE09E
:101A070070109008E4E0C39405A851B800069552F9
:101A1700400280109000AEE0252BFFAE2A50010E49
:101A27008E2A8F2B9008EBE0600D9008E4E0A85118
:101A3700B800069552400280109000AEE0252BFFBB
:101A4700AE2A50010E8E2A8F2B021E0D900086E0C3
:101A5700B402028003021E0D900089E0602FE56743
:101A6700D39446402890000EE0FEA3E0FF9000C408
:101A7700E075F003A4FDACF0EFD39DEE9C400E9013
:101A870000E8E0A851B80005D395525003021E0D97
:101A97009000B9E0B403028003021C5585615A75B2
:101AA7005900900090E0A851B800049552500E904C
:101AB7000091E0A859B80005D3955A5003021C526B
:101AC700E56175F002A4FFAEF074158E048F05FF73
:101AD7001273928C068D0790060E120048FEE0FFE7
:101AE700EE900088E0FEEF8E0088F0A4FFAEF07461
:101AF700648E048F05FF1273928C598D5A9000489B
:101B0700E075F018A4FFAEF09000CFE08E048F05CB
:101B1700FF1273928C068D07900626120048AE5965
:101B2700AF5AE01273A274648E048F05FF1273928A
:101B37008C598D5AE565A859B80005D3955A5003B5
:101B4700021BC9E565C3955AFFE49559FE8E598F67
:101B57005A7428BE00039F500C755A287559007493
:101B67000D900049F0AE59AF5A900089E01273A268
:101B770074288E048F05FF1273928C598D5A900822
:101B870086E0FEA3E0FF740A8E048F05FF127392AE
:101B97008D068C07AC59AD5ACFCECF120003740A0D
:101BA7008E048F05FF1273928C598D5A900886E028
:101BB700FEA3E0FF1273ED900886EEF0A3EFF002AC
:101BC7001C52E565A859B80004955A507EAE59AF26
:101BD7005AE5651273E58E598F5A7428BE00039F24
:101BE700500C755A28755900740D900049F0AE597C
:101BF700AF5A900089E01273A274288E048F05FFF4
:101C07001273928C598D5A900886E0FEA3E0FF74F8
:101C17000A8E048F05FF1273928D068C07AC59AD9F
:101C27005ACFCECF120003740A8E048F05FF1273AA
:101C3700928C598D5A900886E0FEA3E0FFEF2DFDA8
:101C4700EE3CFC900886ECF0A3EDF0021E0D900030
:101C5700D1E0855FF0A4FFAEF074051273A274079C
:101C67001200398E598F5A900090E0A851B800049D
:101C770095525012900091E075F002A4FDACF0EF80
:101C8700C39DEE9C4003021E0DE55F75F00B84FFBC
:101C97007E0090060E120048FEE0FFEE900088E0FE
:101CA700FEEF8E0088F0A4FFAEF074648E048F05FB
:101CB700FF1273928C598D5A900048E075F018A462
:101CC700FFAEF09000CFE08E048F05FF1273928C69
:101CD700068D07900626120048AE59AF5AE01273D8
:101CE700A274648E048F05FF1273928C598D5AE586
:101CF70065A859B80005D3955A5003021D84E565B8
:101D0700C3955AFFE49559FE8E598F5A7428BE0021
:101D1700039F500C755A28755900740D900049F0AF
:101D2700AE59AF5A900089E01273A274288E048FBF
:101D370005FF1273928C598D5A900886E0FEA3E036
:101D4700FF740A8E048F05FF1273928D068C07AC01
:101D570059AD5ACFCECF120003740A8E048F05FFF8
:101D67001273928C598D5A900886E0FEA3E0FF12F9
:101D770073ED900886EEF0A3EFF0021E0DE565A85F
:101D870059B80004955A507EAE59AF5AE56512739B
:101D9700E58E598F5A7428BE00039F500C755A2838
:101DA700755900740D900049F0AE59AF5A900089EB
:101DB700E01273A274288E048F05FF1273928C5958
:101DC7008D5A900886E0FEA3E0FF740A8E048F0503
:101DD700FF1273928D068C07AC59AD5ACFCECF1236
:101DE7000003740A8E048F05FF1273928C598D5A63
:101DF700900886E0FEA3E0FFEF2DFDEE3CFC900887
:101E070086ECF0A3EDF0229000E4E0B4027BE55FFE
:101E170075F00884FF7E008F37E55F75F00884ADA5
:101E2700F07C008D3A753F08755901755AE0E53722
:101E3700C3943F5005121188800690027DE0F53764
:101E4700E537900888F8E4F0E8A3F0900888E0FE0A
:101E5700A3E0FFAC2AAD2B12000374648E048F0538
:101E6700FF127392900888ECF0A3EDF0900081E0E8
:101E77008C068D071273A274648E048F05FF12738C
:101E870092900888ECF0A3EDF0900886E0FEA3E0BE
:101E9700FFAC2AAD2B12000374648E048F05FF126A
:101EA7007392900886ECF0A3EDF0900081E08C0629
:101EB7008D071273A274648E048F05FF12739290BC
:101EC7000886ECF0A3EDF0A204401DAE51AF5274AA
:101ED70005BE00039F5002D204E561D394CC4008AD
:101EE700D2027411900049F0229000E3E0B4020896
:101EF7009000D1E0640B60028045900886E0FEA365
:101F0700E0FFE56B1273A274E78E048F05FF12736F
:101F170092900886ECF0A3EDF09000E4E0B4021F85
:101F2700900888E0FEA3E0FFE56B1273A274E78ECA
:101F3700048F05FF127392900888ECF0A3EDF090E0
:101F470000A3E05402601B90009AE0A851B8001269
:101F5700D39552400DA204B3B35007E561C3949AD9
:101F67004002805FAE34AF35900098E075F002A470
:101F7700FDACF0EF2DFDEE3CFC74022DFD50010C85
:101F8700E561BC003ED39D403A754301A22F403323
:101F9700900099E075F05EA4FDACF07405FF127334
:101FA700928C5B8D5C124B75900886E0FEA3E0FF78
:101FB700900099E02FFF50010E900886EEF0A3EFF6
:101FC700F0D22FE561A834B8000495355002C22F2E
:101FD700856135753400E54370030220E69000F60D
:101FE700E0C3954350030220D8900106E0C3940252
:101FF7004003022082E56775F00A84FF7E009005A2
:102007007E120048E0F55A755900AE59AF5A900054
:1020170099E01273A274648E048F05FF1273928C79
:102027005B8D5C9000F6E004C395438C068D071228
:1020370073A29000F6E08E048F05FF1273928C5BFB
:102047008D5C900886E0FEA3E0FFEF2DFDEE3CFCE3
:10205700900886ECF0A3EDF09000E4E0B4021A904B
:102067000888E0FEA3E0FFAA5BAB5CEF2BFBEE3A30
:10207700FA900888EAF0A3EBF080569000F6E004A7
:10208700C39543854BF0A4FFAEF09000F6E08E04B5
:102097008F05FF1273928C5B8D5C900886E0FEA320
:1020A700E0FFEF2DFDEE3CFC900886ECF0A3EDF091
:1020B7009000E4E0B4021A900888E0FEA3E0FFAACB
:1020C7005BAB5CEF2BFBEE3AFA900888EAF0A3EBE8
:1020D700F005439000F6E0C3954350037543009025
:1020E70000A3E05401601B900097E0A851B80012CC
:1020F700D39552400DA204B3B35007E55FC394CC08
:1021070040028060900095E075F003A4FFAEF0E513
:10211700402FFF50010E74032FFF50010EE55FBEE5
:102127000042D39F403E754401A22F40379000964E
:10213700E075F05EA4FFAEF074058E048F05FF1204
:1021470073928C5B8D5C124B75900886E0FEA3E062
:10215700FF900096E02FFF50010E900886EEF0A347
:10216700EFF0D22FE55FC395405002C22F855F4045
:10217700E54470030222809000F7E0C395445003C2
:10218700022272900106E0C39402400302221CE57A
:102197006775F00A84FF7E0090057E120048E0F51F
:1021A7005A755900AE59AF5A900096E01273A2744F
:1021B700648E048F05FF1273928C5B8D5C9000F721
:1021C700E004C395448C068D071273A29000F7E0D4
:1021D7008E048F05FF1273928C5B8D5C900886E0EE
:1021E700FEA3E0FFEF2DFDEE3CFC900886ECF0A38C
:1021F700EDF09000E4E0B4021A900888E0FEA3E056
:10220700FFAA5BAB5CEF2BFBEE3AFA900888EAF08B
:10221700A3EBF080569000F7E004C39544854CF09B
:10222700A4FFAEF09000F7E08E048F05FF127392C3
:102237008C5B8D5C900886E0FEA3E0FFEF2DFDEE42
:102247003CFC900886ECF0A3EDF09000E4E0B402CB
:102257001A900888E0FEA3E0FFAA5BAB5CEF2BFBBC
:10226700EE3AFA900888EAF0A3EBF005449000F7FD
:10227700E0C395445003754400900886E0FEA3E050
:10228700FF9000A8E0BE00039F500D9000A8E090CB
:102297000886F8E4F0E8A3F09000E4E0B4021290B6
:1022A7000888E0FEA3E0FF9000A8E0BE00059F407D
:1022B70002800D9000A8E0900888F8E4F0E8A3F009
:1022C700229000E4E0B401028003022416A204B3C2
:1022D70050030223FD9000AFE0B4017A900886E036
:1022E700FEA3E0FFAC51AD52120003743C8E048F85
:1022F70005FF1273929000BFE0BC00159D4012903D
:102307000886E0FEA3E0FF9000C1E0BE00039F50F7
:1023170002D203900886E0FEA3E0FFAC51AD521253
:102327000003743C8E048F05FF1273929000BFE088
:10233700C3940ABC001AD39D4016900886E0FEA3FA
:10234700E0FF9000C1E0C39405BE0004D39F500294
:102357008002C203807A900886E0FEA3E0FFAC51BA
:10236700AD5212000374788E048F05FF127392909A
:1023770000BFE0BC00159D4012900886E0FEA3E078
:10238700FF9000C1E0BE00039F5004D2038041903C
:102397000886E0FEA3E0FFAC51AD5212000374784B
:1023A7008E048F05FF1273929000BFE0C3940ABC9E
:1023B700001AD39D4016900886E0FEA3E0FF900028
:1023C700C1E0C39405BE0004D39F50028002C2033C
:1023D700A203B34021900886E0FEA3E0FF9000C06F
:1023E700E01273A274648E048F05FF127392900833
:1023F70086ECF0A3EDF0A203B3400CA233400674C1
:1024070024900049F0D233A2034002C2338002C2B3
:1024170003900044E06006A204B3B3400280199021
:102427000886E0FEA3E0FF900044E02FFF50010E76
:10243700900886EEF0A3EFF0A201B34006A202B324
:10244700B35009900016E4F0A3F0802D900886E0C1
:10245700FEA3E0FF7400D39F74019E40119008868D
:10246700E0F8A3E0900016C8F0A3C8F0800B74FF53
:10247700900016F8E4F0E8A3F09000C6E0C39404D7
:10248700400C9008E8E0C3940240030225709000D6
:10249700AFE0B40147900886E0FEA3E0FF745E1248
:1024A70073A274058E048F05FF127392900886EC51
:1024B700F0A3EDF09000E4E0B4021F900888E0FE7E
:1024C700A3E0FF745E1273A274058E048F05FF12DA
:1024D7007392900888ECF0A3EDF08045900886E0B1
:1024E700FEA3E0FF745E1273A2740A8E048F05FFC9
:1024F700127392900886ECF0A3EDF09000E4E0B43C
:10250700021F900888E0FEA3E0FF745E1273A274B6
:102517000A8E048F05FF127392900888ECF0A3EDE2
:10252700F0900886E0FEA3E0FF7402BE000CD39F84
:102537004008752902752800800A900886E0F5286A
:10254700A3E0F529900888E0FEA3E0FF7402BE002F
:102557000CD39F4008752D02752C00800A900888BF
:10256700E0F52CA3E0F52D8046900886E0FEA3E079
:10257700FF7401BE000CD39F400875290175280020
:10258700800A900886E0F528A3E0F529900888E0FE
:10259700FEA3E0FF7401BE000CD39F4008752D0118
:1025A700752C00800A900888E0F52CA3E0F52D90A3
:1025B7000014E528F0A3E529F0A236B34009C201CB
:1025C700900016E4F0A3F022900048E090037E12FA
:1025D70073D3E0F541754264900048E0FE9000BA7D
:1025E700E0D39E4037E55F75F00884FF7E008F37A4
:1025F700E55F75F00884ADF07C008D3A753F08758E
:102607005903755A96E537C3941F500512118880F0
:1026170006900433E0F5378537428035E55F75F07E
:102627000884FF7E008F37E55F75F00884ADF07C86
:10263700008D3A753F08755903755AB6E537C39447
:102647001F50051211888006900453E0F53785372F
:1026570042229000F0E0F53C753F11755904755A18
:1026670000AE51AF52E53C75F00FA4FDACF0EDD3D1
:102677009FEC9E4021E53C8E048F05FF127392ED7F
:1026870075F010A4FFAEF0E55F75F01184FD7C00D6
:10269700ED2FF53D800EE55F75F01184FF7E00EFAD
:1026A70024F0F53D853D37E55F75F01184AFF07E89
:1026B700008F3A12118885373EAE51AF529000F025
:1026C700E075F00FA4FDACF0EDD39FEC9E402875AC
:1026D7005904755A10853D37121188853E3885375C
:1026E70039AE51AF52E53C8E048F05FF1273BD8D95
:1026F7003A853C3B121202853741754264229000AD
:10270700F0E0F53C753F11755904755A00AE51AFAD
:1027170052E53C75F00FA4FDACF0EDD39FEC9E4065
:1027270021E53C8E048F05FF127392ED75F010A41E
:10273700FFAEF0E56175F01184FD7C00ED2FF53DEE
:10274700800EE56175F01184FF7E00EF24F0F53D02
:10275700853D37E56175F01184AFF07E008F3A1241
:10276700118885373EAE51AF529000F0E075F00FFB
:10277700A4FDACF0EDD39FEC9E4028755904755A23
:1027870010853D37121188853E38853739AE51AFF0
:1027970052E53C8E048F05FF1273BD8D3A853C3B95
:1027A7001212028537417542649000EBE0B4047958
:1027B700900048E0FE9000BAE0D39E4037E55F7591
:1027C700F00884FF7E008F37E55F75F00884ADF071
:1027D7007C008D3A753F08755903755A96E537C3DE
:1027E700941F50051211888006900433E0F5378551
:1027F70037428035E55F75F00884FF7E008F37E547
:102807005F75F00884ADF07C008D3A753F08755907
:1028170003755AB6E537C3941F5005121188800611
:10282700900453E0F53785374222900084E0B401E5
:102837003BE56775F00A84FF7E008F37E56775F023
:102847000A84ADF07C008D3A753F0A755905755AB3
:1028570012E537C39411500512118880069005A11F
:10286700E0F537E5422537C39464F542900085E0EB
:10287700B4013BE56875F00A84FF7E008F37E56891
:1028870075F00A84ADF07C008D3A753F0A755905DD
:10289700755A7EE537C3941150051211888006904A
:1028A700060DE0F537E5422537C39464F542E54167
:1028B7002542F53690008CE0B402109008E0E02540
:1028C70036FE9000E0E0F4042EF5369000E3E0D306
:1028D70094014040E56BC394E7501D74E7C3956BC3
:1028E700FE9008E2E08E00F5F0E884FF7E008F3767
:1028F700E5362537F536801CE56BC394E7FE90086F
:10290700E2E08E00F5F0E884FF7E008F37E536C3FE
:102917009537F536A2044006E5412464F536E536D9
:10292700D394644009E536C39464F536800375365D
:10293700009000BCE0C3953650069000BCE0F53629
:1029470022D20190006CE0A851B800049552503E85
:1029570090006CE0A851B800049552500375360FEB
:1029670090006CE004A851B80004955250037536E6
:102977000790006CE02402A851B800049552500259
:10298700C20190006CE060067409900049F0C22E05
:102997007E017F009000C2E01273A29000D1E08E0A
:1029A700048F05FF127392E55FBC000CD39D4008AE
:1029B700D236740A900049F0900084E0B40109907F
:1029C70000C3E0C39567400280159000D5E0A85189
:1029D700B8000495525002C201740B900049F09060
:1029E7000084E0B40107E567C394644002801D904A
:1029F700011BE0600D90011BE0A851B8000695523D
:102A070040028008C201740B900049F0A201400304
:102A1700753600C235900104E0B40114900105E059
:102A2700A851B8000495525007E55FC3956040026E
:102A3700802A9000ADE0D3941D400B9000ADE0C319
:102A4700941EF5368003753600A23240087415903F
:102A57000049F0D235D232D230022B42C230C232D4
:102A670090008CE0B40306A228B3B34003022B42C4
:102A77009008E4E0C39405A851B8000495525006A5
:102A87009008EBE06002801F9000ADE0D3941D40FA
:102A97000B9000ADE0C3941EF536800375360074C5
:102AA7000C900049F0D2359008E4E0A851B8000432
:102AB700955250069008EBE07002801F9000ADE041
:102AC700D3941D400B9000ADE0C3941EF5368003F0
:102AD700753600740C900049F0D2359008E4E0A8F0
:102AE70051B80004955250319000CBE0B40228D27F
:102AF7002E9008EAE0FE9008EBE0D39E500690087F
:102B0700EBE0700280099008EAE4F0C22E8006909C
:102B170008EAE004F08002C2019008E4E02405A876
:102B270051B80004955250139000CBE0B4020A90BC
:102B370008EBE07002D22E8002C201A22DB340271B
:102B47009000ADE0D3941D400B9000ADE0C3941E00
:102B5700F5368003753600A231400674109000499F
:102B6700F0D231D2358002C23185366C9000ADE0AB
:102B7700D3941D401890007BE02536FE900048E076
:102B870075F01E84FC7F00EE2CF5368029A235B344
:102B9700400890007BE0F536801C90007DE02536EC
:102BA700FE90007BE02EFE900048E075F01E84FC4E
:102BB7007F00EE2CF536A236B34005D22E756C0099
:102BC70022900048E075F00584FF7E008F37900063
:102BD70048E075F00584ADF07C008D3A753F0575CA
:102BE7005903755AD69000CFE01475F00584FF7E1F
:102BF70000E537BE00039F5005121188800BE537AB
:102C07009004541273D3E0F537E5379008E3F0905A
:102C170008E3E0FE9000BEE0C39E50089000BEE0CF
:102C27009008E3F09000ADE0D3941D401E9008E3B8
:102C3700E0FE90007BE02EFE900048E075F01E84D9
:102C4700FC7F00EE2C9008E3F08031A235B3400AF8
:102C570090007BE09008E3F080229008E3E0FE908C
:102C6700007DE02EFE90007BE02EFE900048E07590
:102C7700F01E84FC7F00EE2C9008E3F02290008485
:102C8700E0B40136E56775F00A84FF7E0090057EA3
:102C9700120048E0F546E546D394644010E546C384
:102CA700946475F00F84FF7E008F4680037546009D
:102CB7009000A1E02546F54680069000A1E0F54684
:102CC70022E56775F00A84FF7E0090057E120048B2
:102CD700E0C394694007E567D3946440559000EBDF
:102CE700E0C394035026900880E0FEA3E0FF74043D
:102CF700120039E55F1273A2740F8E048F05FF125D
:102D0700739290087EECF0A3EDF08024900880E0A9
:102D1700FEA3E0FF7404120039E5611273A2740F79
:102D27008E048F05FF12739290087EECF0A3EDF0EE
:102D3700800F900880E0F8A3E090087EC8F0A3C851
:102D4700F0A204401A900880E0FEA3E0FF7403128B
:102D570073A2740112003990087EEEF0A3EFF09091
:102D67000094E0B40262E56AC3944175F00584FFFC
:102D77007E008F37E56A75F00584ADF07C008D3AEB
:102D8700753F05755906755A14E537C394175005ED
:102D970012118880069006A5E0F53790087EE0FEC0
:102DA700A3E0FF740A8E048F05FF127392E5378C38
:102DB700068D071273A2740A8E048F05FF12739291
:102DC70090087EECF0A3EDF090087EE0FEA3E0FF14
:102DD700900884E0FCA3E0FDEDD39FEC9E400F90AC
:102DE7000884E0F8A3E090087EC8F0A3C8F022E5C5
:102DF7000875F004A4FFAEF09006C1120048E090F9
:102E07003C4BF8282873804C85527380479000D13B
:102E1700E0855FF0A4FFAEF074081200398F73806D
:102E270033856173802E8567738029856873802455
:102E3700856973801F856A73801A856B7380158512
:102E470066738010856573800B856C7380069000B0
:042E570017E0F57318
:103C4B00022E0D022E0F022E14022E28022E2D02F2
:103C5B002E32022E37022E3C022E41022E46022E0F
:073C6B004B022E50022E5502
:102E5B00E50875F004A4FFAEF09006C2120048E539
:102E6B000875F004A4FFAEF0E0FC9006C312004816
:102E7B00ECFEE0FFEEC39F4003022F63E50875F005
:102E8B0004A4FFAEF09006C1120048E0B40441E583
:102E9B000875F004A4FFAEF09006C3120048E0C31F
:102EAB009573500AE508F50CD39237123DF0E508FF
:102EBB0075F004A4FFAEF09006C2120048E0D39563
:102ECB0073400AE508F50CC39237123DF0022F61EF
:102EDB00E50875F004A4FFAEF09006C2120048E0BE
:102EEB00C395735015E50875F004A4FFAEF090067A
:102EFB00C3120048E0D395735002800AE508F50C25
:102F0B00D39237123DF0E50875F004A4FFAEF090B4
:102F1B0006C2120048E0D395735015E50875F0040E
:102F2B00A4FFAEF09006C3120048E0C39573500A9D
:102F3B00E508F50CC39237123DF09006C9E0B401D9
:102F4B00099000DDE0D395615002800A7402F50C04
:102F5B00C39237123DF0806AE50875F004A4FFAE0A
:102F6B00F09006C2120048E0D395734015E5087542
:102F7B00F004A4FFAEF09006C3120048E0C39573B3
:102F8B004002800AE508F50CC39237123DF0E508C4
:102F9B0075F004A4FFAEF09006C2120048E0C39592
:102FAB00734015E50875F004A4FFAEF09006C3124C
:102FBB000048E0D39573400AE508F50CD39237121D
:102FCB003DF022AE2EAF2F74C9BE000CD39F40082C
:102FDB00782E1273F50230E8752F01752E00AE5165
:102FEB00AF52E546BE000DD39F40099000B3E0D32E
:102FFB00954740028023754700E546C39552F5730C
:10300B009000B6E0D395454008E5452573F545801E
:10301B00069000B6E0F5458002054790008FE0D39F
:10302B009561401CE55FC395604015AE51AF52E50D
:10303B0046BE00039F50099000B4E0D39548400270
:10304B00806E9008E5E0A851B800049552500375C6
:10305B004A009008E5E0A851B8000BD39552400602
:10306B00E5529008E5F0E54A7041E552C39546F507
:10307B0073E573D3940540037573059000B5E0C3F6
:10308B0095455007E573C3954540028009E545C357
:10309B009573F54580069000B5E0F5459000B5E0D9
:1030AB00D3954540069000B5E0F545754800800284
:1030BB000548E54A701690008FE0C39561500DE509
:1030CB00462405A851B8000695524002800F900087
:1030DB00A2E0F545754A0174789008E5F022AE2E12
:1030EB00AF2F74E9D39F74039E4008782E1273F5AB
:1030FB0002328F752F01752E00754532A229402A99
:10310B007545199000A2E075F002A4FFAEF0E547FB
:10311B00BE0006D39F4002D2290547754A03747837
:10312B009008E5F0754900023276AE51AF52E54694
:10313B006F4E7003023276E546BE000DD39F4009F9
:10314B009000B3E0D395474002800F754700E54AE6
:10315B00C394035003754519800DE546C39552F58D
:10316B0073E5472573F54790008FE0D39561400ECB
:10317B009008E5E0A851B80007D395524002800CA7
:10318B0005499000A2E0B54903754A00E54AB4032E
:10319B0006A204B3B34002800A0549E549B43C03D7
:1031AB00754A02E54AB402299008E5E0A851B80037
:1031BB000ED395524009E5529008E5F07549009001
:1031CB00008FE0C39561500975490074789008E54C
:1031DB00F0E54A705A90008FE0D39561401CE55F93
:1031EB00C395604015AE51AF52E546BE00039F50EC
:1031FB00099000B4E0D395484002800875480075EB
:10320B00454B8028E552C39546F573E573D394057A
:10321B00400375730590008FE0D395614008E54836
:10322B002573F5488006E5482406F548754900E501
:10323B004A701690008FE0C39561500DE54624054A
:10324B00A851B80006955240028003754A01E54A21
:10325B00B4011875451905499000A2E0B5490675EA
:10326B004A0275490074789008E5F0A202B3400356
:10327B00754532E54575F00AA4FFAEF090088AEE6D
:10328B00F0A3EFF022E56F903C72F8282873023C14
:10329B000B900087E070030235BA9000BDE0B401DB
:1032AB00028003023450900046E0655E6009E552EF
:1032BB004551600302344D7E017F00E5BE1273A2BF
:1032CB00E5BD2FFF50010E8E598F5A9000BBE0B415
:1032DB00461B740E1273A290006BE08E048F05FFD9
:1032EB0012739290088EECF0A3EDF0801DAE59AFE7
:1032FB005A74101273A290006BE08E048F05FF12AC
:10330B00739290088EECF0A3EDF0E56B600FE56B1C
:10331B00C394FE50089000E3E06402600280649066
:10332B0000D1E0B40B1F90088EE0FEA3E0FF74E722
:10333B001273A2E56B8E048F05FF12739290088EA9
:10334B00ECF0A3EDF09000D1E0D3940B400890008B
:10335B00B9E064046002802B90088EE0FEA3E0FFCE
:10336B00900892E0FCA3E0FDEFD39DEE9C400D1284
:10337B0073ED90088EEEF0A3EFF0800790088EE4CB
:10338B00F0A3F090088EE0FEA3E0FFEFD39400EEE5
:10339B0094014008D2367426900049F0A236B3B39C
:1033AB00502C7E057F009000D1E08E048F05FF121C
:1033BB00739290088EE0FEA3E0FFEFC39DEE9C405E
:1033CB000FAC51AD52740FBC0004D39D5002800260
:1033DB00C236900087E0B40227900890E0FEA3E08D
:1033EB00FF90088EE0FCA3E0FDEF2DFDEE3CFC749E
:1033FB00018C068D0712003990088EEEF0A3EFF0CA
:10340B0090088EE0FEA3E0FF900890E0FCA3E0FDA7
:10341B00EDD39FEC9E4004D22C8002B22C90088EF0
:10342B00E0F8A3E0900890C8F0A3C8F09000B9E0D2
:10343B0064016006A22CB3B34002800690088FE0B3
:10344B00F55F0235B8D22C7E017F00E5BE1273A268
:10345B00E5BD2FFF50010E8E598F5A9000BBE0B483
:10346B00461B740E1273A290006BE08E048F05FF47
:10347B0012739290088EECF0A3EDF0801DAE59AF55
:10348B005A74101273A290006BE08E048F05FF121A
:10349B00739290088EECF0A3EDF0E56B600FE56B8B
:1034AB00C394FE50089000E3E064026002806490D5
:1034BB0000D1E0B40B1F90088EE0FEA3E0FF74E791
:1034CB001273A2E56B8E048F05FF12739290088E18
:1034DB00ECF0A3EDF09000D1E0D3940B40089000FA
:1034EB00B9E064046002802B90088EE0FEA3E0FF3D
:1034FB00900892E0FCA3E0FDEFD39DEE9C400D12F3
:10350B0073ED90088EEEF0A3EFF0800790088EE439
:10351B00F0A3F090088EE0FEA3E0FFEFD39400EE53
:10352B0094014008D2367426900049F0A236B3B30A
:10353B00502C7E057F009000D1E08E048F05FF128A
:10354B00739290088EE0FEA3E0FFEFC39DEE9C40CC
:10355B000FAC51AD52740FBC0004D39D50028002CE
:10356B00C236900087E0B40227900890E0FEA3E0FB
:10357B00FF90088EE0FCA3E0FDEF2DFDEE3CFC740C
:10358B00018C068D0712003990088EEEF0A3EFF038
:10359B0090088EE0F8A3E0900890C8F0A3C8F090D4
:1035AB0000B9E06401600690088FE0F55F80037559
:1035BB005F00900083E07006756F0302329075BB5D
:1035CB0018023C0B023C0B900083E0700302374364
:1035DB007E017F00E5BE1273A2E5BD2FFF50010EE9
:1035EB008E598F5A9000C9E0B4010F7E0F7FFFAC4C
:1035FB0059AD5A1273ED8E598F5A9000EEE0B4020A
:10360B0045AE59AF5A900020E0FCA3E0FDEDD39FEF
:10361B00EC9E400A900020E559F0A3E55AF0AE5914
:10362B00AF5A900022E0FCA3E0FDEFD39DEE9C404F
:10363B000A900022E559F0A3E55AF0AE59AF5A743F
:10364B00041200398F619000EEE0704CAE59AF5A06
:10365B00900020E0FCA3E0FDEFD39DEE9C4009120F
:10366B0073ED8E598F5A8006755A00755900AE59F5
:10367B00AF5A74101273A29000EDE08E048F05FF09
:10368B001273928C598D5A74FFBC0009D39D40055F
:10369B00855A6180037561FE9000B9E0B401028028
:1036AB0003023741A204B3B3500E90008DE0A85132
:1036BB00B80005D39552500280719000CAE0856125
:1036CB00F0A4FFAEF074648E048F05FF1273928C1E
:1036DB00598D5AE56B6016E56BC394FE500F900045
:1036EB00E3E0B402089000D1E0640B60028017AEF7
:1036FB0059AF5A74E71273A2E56B8E048F05FF1254
:10370B0073928C598D5AAE59AF5A90088EE0FCA328
:10371B00E0FDEDD39FEC9E4005855A5F800BA22CFC
:10372B00B3400690088FE0F55F800BA22CB34006E8
:10373B0090088FE0F55F8003756100900086E07064
:10374B0006756F0502329075BB19023C0B023C0BE0
:10375B00900086E070030237FBE55ED3955D400376
:10376B000237F990001EE0FEA3E0FFE5651273E55A
:10377B0090001EEEF0A3EFF07E017F00E5BE12730A
:10378B00A2E5BD2FFF50010E8E598F5A9000F3E02A
:10379B007013740A1273A274518E048F05FF127387
:1037AB00928D658019AE59AF5A740A1273A28F04A9
:1037BB008E057E017F95CDCCCD1272908F65E56520
:1037CB00D39464400375656490001EE0FEA3E0FF94
:1037DB00E5652FFF50010E90001EEEF0A3EFF09069
:1037EB00008AE0048E048F05FF1273928D658003AF
:1037FB007565329000D6E07006756F0702329075D2
:10380B00BB13023C0B023C0B9000D6E0604A7E01DE
:10381B007F00E5BE1273A2E5BD2FFF50010E8E593E
:10382B008F5A74041200398F669000D8E08566F0C9
:10383B00A4FDACF07464FF1273928D669000D7E018
:10384B008566F0A4FFAEF074FF8E048F05FF127334
:10385B0092ED90006AF08003756600900084E07032
:10386B0006756F0902329075BB17023C0B023C0BBD
:10387B00900084E0B40102800302390F7E017F00C7
:10388B00E5BE1273A2E5BD2FFF50010E8E598F5A64
:10389B009008E6E060199008E6E014906D82120043
:1038AB008CE493FC740193FDEDC39FEC9E4002806E
:1038BB00069008E6E014F09008E6E0C394B3501DC0
:1038CB00AE59AF5A9008E6E004906D8212008CE47A
:1038DB0093FC740193FDEFC39DEE9C400280069018
:1038EB0008E6E004F09008E6E0FE9000AAE08E0007
:1038FB0088F0A4FFAEF074648E048F05FF127392F0
:10390B008D678003756700900085E07006756F0BFF
:10391B0002329075BB16023C0B023C0B900085E00B
:10392B00B4010280030239BB7E017F00E5BE127336
:10393B00A2E5BD2FFF50010E8E598F5A9008E7E07C
:10394B0060199008E7E014906EEC12008CE493FC85
:10395B00740193FDEDC39FEC9E400280069008E737
:10396B00E014F09008E7E0C394B3501DAE59AF5A82
:10397B009008E7E004906EEC12008CE493FC740169
:10398B0093FDEFC39DEE9C400280069008E7E00498
:10399B00F09008E7E0FE9000B0E08E0088F0A4FF06
:1039AB00AEF074648E048F05FF1273928D688003E2
:1039BB0075680075BB1F023C0B023C0B7E017F0040
:1039CB00E5BE1273A2E5BD2FFF50010E8E598F5A23
:1039DB0074091273A274E68E048F05FF1273928D15
:1039EB006A90008CE07006756F0F02329075BB15F4
:1039FB00023C0B023C0B90008CE07003023B527EAE
:103A0B00017F00E5BE1273A2E5BD2FFF50010E8EA4
:103A1B00598F5A74041200398F6990008CE0B401ED
:103A2B00159000E0E08569F0A4FFAEF0740712007A
:103A3B0039EF9008E1F090008CE0B402159000E0B3
:103A4B00E08569F0A4FFAEF07407120039EF90081F
:103A5B00E0F090008CE0B403028003023B35900051
:103A6B00CDE07052E569C39419500FD2289000AC89
:103A7B00E09008E4F09008E9E4F0E569D394644041
:103A8B0004A2284002802D9008E9E004F09008E998
:103A9B00E0FE90011FE0B5060B9008E4E004F09007
:103AAB0008E9E4F09008E4E06496600690011FE0FA
:103ABB007002C22880639000ACE070349000E0E0AC
:103ACB008569F0A4FFAEF074FF8E048F05FF1273AF
:103ADB0092ED9008E4F0AE51AF52741EBE0006D3C7
:103AEB009F4002D228E561D394E54002C228802989
:103AFB00E569C3940A500DAE51AF52741EBE00045B
:103B0B00D39F50028002D228E561D394E54002C2D4
:103B1B00289000ACE09008E4F09008E4E0C3940532
:103B2B00500674059008E4F0C22D90008CE0B404AC
:103B3B0014E569C394195002D22DE569D394324030
:103B4B0002C22DC22880037569009000E3E0700665
:103B5B00756F1102329075BB14023C0B023C0B903B
:103B6B0000E3E07003023BF87E017F00E5BE1273B9
:103B7B00A2E5BD2FFF50010E8E598F5A900108E020
:103B8B007025EFD39421EE940E4005756BFF8015D5
:103B9B00AE59AF5A74101273A274E38E048F05FFE3
:103BAB001273928D6B8027AE59AF5AEFD39449EEB7
:103BBB0094064005756BFF8015AE59AF5A74101201
:103BCB0073A274638E048F05FF1273928D6BE56B7A
:103BDB0075F00BA4FFAEF09000D1E08E048F05FFC3
:103BEB00127392900892ECF0A3EDF08003756B00CA
:103BFB00900087E0600575BB1A800375BB188000C9
:103C720002329902329C0235CF0235D20237580203
:103C8200375B02381002381302387802387B023967
:103C9200240239270239C40239C70239FE023A0125
:093CA200023B67023B6A023C0B85
:103C0B00E56F75F00284AFF07E00EF4E7002D2ECE0
:033C1B00056F2210
:0973D3002582F582500205832297
:0F008C0025E050020583258250020583F582226C
:10737100EF2F500205832582F582E5833E2EF583AA
:0173810022E9
:1073E500CFC39FFF50011E22C3EF9DFFEE9CFE22DF
:0873F5000806B600021806228A
:0D73B000A3E004F070061273C9E004F0229F
:0E003900048007C3CE13CECF13CFD5E0F6223E
:10729000BC000FBE0008ED8FF084FFADF022E4FECD
:1072A000FF22BE000DEF60FE54F0606F20E7030286
:1072B0007346EAC0E0EBC0E078017A0075F001EEB9
:1072C00020E710EF25E0FFEE33FE0AC5F023C5F0FE
:1072D00030E7F0EA5407F9096A7A007B0060010898
:1072E000C3EC9E40167004ED9F4010ED9FFDEC9E98
:1072F000FCE5F0CA4ACA03F5F08005E5F003F5F0B5
:10730000C3EE13FEEF13FFD9D77908CACBCAD8D082
:10731000EAFEEBFFD0E0FBD0E0FA22EC8FF084FC39
:10732000ED54F045F0C48FF084FEEDC454F045F008
:10733000C48FF084FDEEC4FE54F02DFFEE540F3CDC
:10734000FEADF07C0022790078008FF0EC7E082002
:10735000E70DC3CD33CD33C933C9C833C8DEF0849C
:1073600049F9E5F08FF0BE00E6FD7C00E9FFE8FE9C
:0173700022FA
:0E73A200F88FF0A4FFE5F0CE88F0A42EFE22B6
:10000300EF8DF0A4F9A8F0EF8CF0A428F8EE8DF0B2
:06001300A428FEE9FF2213
:10738200600D782B02738C007830D8FED5E0F8229D
:10739200EEC0E07E00127290EFFDEEFCD0E0FE2225
:0C73BD00EEC0E07E00127290D0E0FE22D4
:03001B0002001EC2
:0300530002005652
:03009B00020071EF
:030000000273DCAC
:0973DC0075817575D000024CDECC
:0B004800E5822FF582E5833EF5832260
:0A73C9000582D58202158315822289
:10001E00C0E0C0F0C083C082C0D075D000124C4882
:0B002E00D0D0D082D083D0F0D0E032E0
:10005600C0E0C0F0C083C082C0D075D000124C4B47
:10006600D0D0D082D083D0F0D0E032C0E0C0F0C093
:1000760083C082C0D075D000124CA0D0D0D082D020
:0600860083D0F0D0E0324F
:00000001FF
